 attach039Agent00

 Timestamp is 0b790713 (reproducible build file hash)

 Preferred load address is 0000000180000000

 Start         Length     Name                   Class
 0001:00000000 00004120H .text$mn                CODE
 0001:00004120 00000036H .text$mn$00             CODE
 0001:00004156 00000092H .text$x                 CODE
 0002:00000000 000001b8H .idata$5                DATA
 0002:000001b8 00000038H .00cfg                  DATA
 0002:000001f0 00000008H .CRT$XCA                DATA
 0002:000001f8 00000008H .CRT$XCZ                DATA
 0002:00000200 00000008H .CRT$XIA                DATA
 0002:00000208 00000008H .CRT$XIC                DATA
 0002:00000210 00000008H .CRT$XIZ                DATA
 0002:00000218 00000008H .CRT$XLA                DATA
 0002:00000220 00000008H .CRT$XLZ                DATA
 0002:00000228 00000008H .CRT$XPA                DATA
 0002:00000230 00000008H .CRT$XPZ                DATA
 0002:00000238 00000008H .CRT$XTA                DATA
 0002:00000240 00000010H .CRT$XTZ                DATA
 0002:00000248 00000000H .gehcont$y              DATA
 0002:00000248 00000000H .gfids$y                DATA
 0002:00000250 000026b0H .rdata                  DATA
 0002:00002900 00000000H .rdata$CastGuardVftablesA DATA
 0002:00002900 00000000H .rdata$CastGuardVftablesC DATA
 0002:00002900 00000028H .rdata$T                DATA
 0002:00002928 000000c0H .rdata$voltmd           DATA
 0002:000029e8 00000320H .rdata$zzzdbg           DATA
 0002:00002d08 00000008H .rtc$IAA                DATA
 0002:00002d10 00000008H .rtc$IZZ                DATA
 0002:00002d18 00000008H .rtc$TAA                DATA
 0002:00002d20 00000008H .rtc$TZZ                DATA
 0002:00002d28 00000004H .tls                    DATA
 0002:00002d2c 00000004H .tls$                   DATA
 0002:00002d30 00000008H .tls$ZZZ                DATA
 0002:00002d38 000003f8H .xdata                  DATA
 0002:00003130 00000354H .edata                  DATA
 0002:00003484 00000078H .idata$2                DATA
 0002:000034fc 00000014H .idata$3                DATA
 0002:00003510 000001b8H .idata$4                DATA
 0002:000036c8 0000045aH .idata$6                DATA
 0003:00000000 000000b0H .data                   DATA
 0003:000000b0 0001b308H .bss                    DATA
 0004:00000000 00000468H .pdata                  DATA

  Address         Publics by Value              Rva+Base               Lib:Object

 0000:00000000       __AbsoluteZero             0000000000000000     <absolute>
 0000:00000000       ___safe_se_handler_count   0000000000000000     <absolute>
 0000:00000000       ___safe_se_handler_table   0000000000000000     <absolute>
 0000:00000000       __arm64x_extra_rfe_table   0000000000000000     <absolute>
 0000:00000000       __arm64x_extra_rfe_table_size 0000000000000000     <absolute>
 0000:00000000       __arm64x_native_entrypoint 0000000000000000     <absolute>
 0000:00000000       __arm64x_redirection_metadata 0000000000000000     <absolute>
 0000:00000000       __arm64x_redirection_metadata_count 0000000000000000     <absolute>
 0000:00000000       __dynamic_value_reloc_table 0000000000000000     <absolute>
 0000:00000000       __enclave_config           0000000000000000     <absolute>
 0000:00000000       __guard_check_icall_a64n_fptr 0000000000000000     <absolute>
 0000:00000000       __guard_eh_cont_count      0000000000000000     <absolute>
 0000:00000000       __guard_eh_cont_table      0000000000000000     <absolute>
 0000:00000000       __guard_fids_count         0000000000000000     <absolute>
 0000:00000000       __guard_fids_table         0000000000000000     <absolute>
 0000:00000000       __guard_iat_count          0000000000000000     <absolute>
 0000:00000000       __guard_iat_table          0000000000000000     <absolute>
 0000:00000000       __guard_longjmp_count      0000000000000000     <absolute>
 0000:00000000       __guard_longjmp_table      0000000000000000     <absolute>
 0000:00000000       __hybrid_auxiliary_iat     0000000000000000     <absolute>
 0000:00000000       __hybrid_auxiliary_iat_copy 0000000000000000     <absolute>
 0000:00000000       __hybrid_code_map          0000000000000000     <absolute>
 0000:00000000       __hybrid_code_map_count    0000000000000000     <absolute>
 0000:00000000       __x64_code_ranges_to_entry_points 0000000000000000     <absolute>
 0000:00000000       __x64_code_ranges_to_entry_points_count 0000000000000000     <absolute>
 0000:00000100       __guard_flags              0000000000000100     <absolute>
 0000:00000000       __ImageBase                0000000180000000     <linker-defined>
 0001:00000000       ?CallStaticVoidMethod@JNIEnv_@@QEAAXPEAV_jclass@@PEAU_jmethodID@@ZZ 0000000180001000 f i libattach039Agent00.obj
 0001:00000024       ?NewObject@JNIEnv_@@QEAAPEAV_jobject@@PEAV_jclass@@PEAU_jmethodID@@ZZ 0000000180001024 f i libattach039Agent00.obj
 0001:0000004c       ?SetEventNotificationMode@_jvmtiEnv@@QEAA?AW4jvmtiError@@W4jvmtiEventMode@@W4jvmtiEvent@@PEAV_jobject@@ZZ 000000018000104c f i libattach039Agent00.obj
 0001:00000058       ?TranslateError@@YAPEBDW4jvmtiError@@@Z 0000000180001058 f   libattach039Agent00.obj
 0001:00000310       ?nsk_jni_check_exception@@YAHPEAUJNIEnv_@@QEBDH@Z 0000000180001310 f   libattach039Agent00.obj
 0001:00000454       ?nsk_jni_lverify@@YAHHPEAUJNIEnv_@@HQEBDH1ZZ 0000000180001454 f   libattach039Agent00.obj
 0001:000004f4       Agent_OnAttach             00000001800014f4 f   libattach039Agent00.obj
 0001:000007a4       Java_nsk_jvmti_unit_FollowReferences_FollowRefObjects_addRefToVerify 00000001800017a4 f   libattach039Agent00.obj
 0001:0000097c       Java_nsk_jvmti_unit_FollowReferences_FollowRefObjects_getTag 000000018000197c f   libattach039Agent00.obj
 0001:00000a3c       Java_nsk_jvmti_unit_FollowReferences_FollowRefObjects_resetRefsToVerify 0000000180001a3c f   libattach039Agent00.obj
 0001:00000a44       Java_nsk_jvmti_unit_FollowReferences_FollowRefObjects_resetTags 0000000180001a44 f   libattach039Agent00.obj
 0001:00000a88       Java_nsk_jvmti_unit_FollowReferences_FollowRefObjects_setTag 0000000180001a88 f   libattach039Agent00.obj
 0001:00000ce0       Java_nsk_share_jvmti_ArgumentHandler_getAgentOptionsString 0000000180001ce0 f   libattach039Agent00.obj
 0001:00000d90       Java_nsk_share_jvmti_DebugeeClass_checkStatus 0000000180001d90 f   libattach039Agent00.obj
 0001:00000e18       Java_nsk_share_jvmti_DebugeeClass_resetAgentData 0000000180001e18 f   libattach039Agent00.obj
 0001:00000e78       Java_nsk_share_jvmti_RedefineAgent_agentStatus 0000000180001e78 f   libattach039Agent00.obj
 0001:00000e84       Java_nsk_share_jvmti_RedefineAgent_isRedefined 0000000180001e84 f   libattach039Agent00.obj
 0001:00000e90       Java_nsk_share_jvmti_RedefineAgent_redefineAttempted 0000000180001e90 f   libattach039Agent00.obj
 0001:00000e9c       MA_checkStatus             0000000180001e9c f   libattach039Agent00.obj
 0001:00000f40       __local_stdio_printf_options 0000000180001f40 f i libattach039Agent00.obj
 0001:00001120       exitOnError                0000000180002120 f   libattach039Agent00.obj
 0001:000011d4       fprintf                    00000001800021d4 f i libattach039Agent00.obj
 0001:00001218       nsk_aod_agentFinished      0000000180002218 f   libattach039Agent00.obj
 0001:00001414       nsk_aod_agentLoaded        0000000180002414 f   libattach039Agent00.obj
 0001:000016e4       nsk_aod_createJNIEnv       00000001800026e4 f   libattach039Agent00.obj
 0001:0000175c       nsk_aod_createOptions      000000018000275c f   libattach039Agent00.obj
 0001:000019cc       nsk_aod_getOptionValue     00000001800029cc f   libattach039Agent00.obj
 0001:00001ab8       nsk_aod_internal_error     0000000180002ab8 f   libattach039Agent00.obj
 0001:00001ae4       nsk_aod_optionSpecified    0000000180002ae4 f   libattach039Agent00.obj
 0001:00001bac       nsk_free_options           0000000180002bac f   libattach039Agent00.obj
 0001:00001c0c       nsk_jvmti_aod_createThreadWithName 0000000180002c0c f   libattach039Agent00.obj
 0001:00001ec0       nsk_jvmti_aod_deallocate   0000000180002ec0 f   libattach039Agent00.obj
 0001:00001f78       nsk_jvmti_aod_disableEvents 0000000180002f78 f   libattach039Agent00.obj
 0001:00002048       nsk_jvmti_aod_disableEventsAndFinish 0000000180003048 f   libattach039Agent00.obj
 0001:00002084       nsk_jvmti_aod_enableEvents 0000000180003084 f   libattach039Agent00.obj
 0001:00002144       nsk_jvmti_aod_getThreadName 0000000180003144 f   libattach039Agent00.obj
 0001:00002228       nsk_jvmti_createJVMTIEnv   0000000180003228 f   libattach039Agent00.obj
 0001:00002358       nsk_jvmti_lverify          0000000180003358 f   libattach039Agent00.obj
 0001:00002448       nsk_jvmti_resetAgentData   0000000180003448 f   libattach039Agent00.obj
 0001:000024c8       nsk_jvmti_setFailStatus    00000001800034c8 f   libattach039Agent00.obj
 0001:00002504       nsk_lcomplain              0000000180003504 f   libattach039Agent00.obj
 0001:00002524       nsk_ldisplay               0000000180003524 f   libattach039Agent00.obj
 0001:00002544       nsk_ltrace                 0000000180003544 f   libattach039Agent00.obj
 0001:00002564       nsk_lvcomplain             0000000180003564 f   libattach039Agent00.obj
 0001:0000271c       nsk_lvdisplay              000000018000371c f   libattach039Agent00.obj
 0001:00002768       nsk_lverify                0000000180003768 f   libattach039Agent00.obj
 0001:000027c4       nsk_lvtrace                00000001800037c4 f   libattach039Agent00.obj
 0001:00002824       nsk_printf                 0000000180003824 f   libattach039Agent00.obj
 0001:0000284c       nsk_vprintf                000000018000384c f   libattach039Agent00.obj
 0001:00002900       printf                     0000000180003900 f i libattach039Agent00.obj
 0001:00002c90       startNewThread             0000000180003c90 f   libattach039Agent00.obj
 0001:00002dc0       startedThreadFunction      0000000180003dc0 f   libattach039Agent00.obj
 0001:00003008       threadEndHandler           0000000180004008 f   libattach039Agent00.obj
 0001:00003120       threadStartHandler         0000000180004120 f   libattach039Agent00.obj
 0001:000031e8       __raise_securityfailure    00000001800041e8 f   MSVCRT:gs_report.obj
 0001:0000321c       __report_gsfailure         000000018000421c f   MSVCRT:gs_report.obj
 0001:0000345c       __GSHandlerCheck           000000018000445c f   MSVCRT:gshandler.obj
 0001:0000347c       __GSHandlerCheckCommon     000000018000447c f   MSVCRT:gshandler.obj
 0001:000034f0       __security_check_cookie    00000001800044f0 f   MSVCRT:amdsecgs.obj
 0001:00003830       _DllMainCRTStartup         0000000180004830 f   MSVCRT:dll_dllmain.obj
 0001:00003870       __scrt_acquire_startup_lock 0000000180004870 f   MSVCRT:utility.obj
 0001:000038ac       __scrt_dllmain_after_initialize_c 00000001800048ac f   MSVCRT:utility.obj
 0001:000038e0       __scrt_dllmain_before_initialize_c 00000001800048e0 f   MSVCRT:utility.obj
 0001:000038f8       __scrt_dllmain_crt_thread_attach 00000001800048f8 f   MSVCRT:utility.obj
 0001:00003920       __scrt_dllmain_crt_thread_detach 0000000180004920 f   MSVCRT:utility.obj
 0001:00003938       __scrt_dllmain_exception_filter 0000000180004938 f   MSVCRT:utility.obj
 0001:00003998       __scrt_dllmain_uninitialize_c 0000000180004998 f   MSVCRT:utility.obj
 0001:000039c8       __scrt_dllmain_uninitialize_critical 00000001800049c8 f   MSVCRT:utility.obj
 0001:000039dc       __scrt_initialize_crt      00000001800049dc f   MSVCRT:utility.obj
 0001:00003a28       __scrt_initialize_onexit_tables 0000000180004a28 f   MSVCRT:utility.obj
 0001:00003ab4       __scrt_is_nonwritable_in_current_image 0000000180004ab4 f   MSVCRT:utility.obj
 0001:00003b4c       __scrt_release_startup_lock 0000000180004b4c f   MSVCRT:utility.obj
 0001:00003b70       __scrt_uninitialize_crt    0000000180004b70 f   MSVCRT:utility.obj
 0001:00003b9c       _onexit                    0000000180004b9c f   MSVCRT:utility.obj
 0001:00003bd8       atexit                     0000000180004bd8 f   MSVCRT:utility.obj
 0001:00003bf0       __crt_debugger_hook        0000000180004bf0 f   MSVCRT:utility_desktop.obj
 0001:00003bf8       __scrt_fastfail            0000000180004bf8 f   MSVCRT:utility_desktop.obj
 0001:00003d44       _guard_check_icall_nop     0000000180004d44 f i MSVCRT:guard_support.obj
 0001:00003d48       __security_init_cookie     0000000180004d48 f   MSVCRT:gs_support.obj
 0001:00003df4       DllMain                    0000000180004df4 f   MSVCRT:dll_dllmain_stub.obj
 0001:00003e18       ?__scrt_initialize_type_info@@YAXXZ 0000000180004e18 f   MSVCRT:tncleanup.obj
 0001:00003e28       ?__scrt_uninitialize_type_info@@YAXXZ 0000000180004e28 f   MSVCRT:tncleanup.obj
 0001:00003e34       __local_stdio_scanf_options 0000000180004e34 f i MSVCRT:default_local_stdio_options.obj
 0001:00003e3c       __scrt_initialize_default_local_stdio_options 0000000180004e3c f   MSVCRT:default_local_stdio_options.obj
 0001:00003e58       __scrt_get_dyn_tls_init_callback 0000000180004e58 f   MSVCRT:dyn_tls_init.obj
 0001:00003e60       _RTC_Initialize            0000000180004e60 f   MSVCRT:initsect.obj
 0001:00003e9c       _RTC_Terminate             0000000180004e9c f   MSVCRT:initsect.obj
 0001:00003ed8       __isa_available_init       0000000180004ed8 f   MSVCRT:cpu_disp.obj
 0001:00004084       _get_startup_argv_mode     0000000180005084 f   MSVCRT:argv_mode.obj
 0001:0000408c       __scrt_is_ucrt_dll_in_use  000000018000508c f   MSVCRT:ucrt_detection.obj
 0001:000040a0       memcpy                     00000001800050a0 f   vcruntime:VCRUNTIME140.dll
 0001:000040a6       memset                     00000001800050a6 f   vcruntime:VCRUNTIME140.dll
 0001:000040ac       strchr                     00000001800050ac f   vcruntime:VCRUNTIME140.dll
 0001:000040b2       __C_specific_handler       00000001800050b2 f   vcruntime:VCRUNTIME140.dll
 0001:000040b8       __std_type_info_destroy_list 00000001800050b8 f   vcruntime:VCRUNTIME140.dll
 0001:000040be       strcmp                     00000001800050be f   ucrt:api-ms-win-crt-string-l1-1-0.dll
 0001:000040c4       strcpy                     00000001800050c4 f   ucrt:api-ms-win-crt-string-l1-1-0.dll
 0001:000040ca       strlen                     00000001800050ca f   ucrt:api-ms-win-crt-string-l1-1-0.dll
 0001:000040d0       _initterm                  00000001800050d0 f   ucrt:api-ms-win-crt-runtime-l1-1-0.dll
 0001:000040d6       _initterm_e                00000001800050d6 f   ucrt:api-ms-win-crt-runtime-l1-1-0.dll
 0001:000040dc       _seh_filter_dll            00000001800050dc f   ucrt:api-ms-win-crt-runtime-l1-1-0.dll
 0001:000040e2       _configure_narrow_argv     00000001800050e2 f   ucrt:api-ms-win-crt-runtime-l1-1-0.dll
 0001:000040e8       _initialize_narrow_environment 00000001800050e8 f   ucrt:api-ms-win-crt-runtime-l1-1-0.dll
 0001:000040ee       _initialize_onexit_table   00000001800050ee f   ucrt:api-ms-win-crt-runtime-l1-1-0.dll
 0001:000040f4       _register_onexit_function  00000001800050f4 f   ucrt:api-ms-win-crt-runtime-l1-1-0.dll
 0001:000040fa       _execute_onexit_table      00000001800050fa f   ucrt:api-ms-win-crt-runtime-l1-1-0.dll
 0001:00004100       _crt_atexit                0000000180005100 f   ucrt:api-ms-win-crt-runtime-l1-1-0.dll
 0001:00004106       _cexit                     0000000180005106 f   ucrt:api-ms-win-crt-runtime-l1-1-0.dll
 0001:0000410c       __acrt_initialize          000000018000510c f   MSVCRT:ucrt_stubs.obj
 0001:0000410c       __acrt_thread_attach       000000018000510c f   MSVCRT:ucrt_stubs.obj
 0001:0000410c       __acrt_thread_detach       000000018000510c f   MSVCRT:ucrt_stubs.obj
 0001:0000410c       __acrt_uninitialize        000000018000510c f   MSVCRT:ucrt_stubs.obj
 0001:0000410c       __acrt_uninitialize_critical 000000018000510c f   MSVCRT:ucrt_stubs.obj
 0001:0000410c       __scrt_stub_for_acrt_initialize 000000018000510c f   MSVCRT:ucrt_stubs.obj
 0001:0000410c       __scrt_stub_for_acrt_thread_attach 000000018000510c f   MSVCRT:ucrt_stubs.obj
 0001:0000410c       __scrt_stub_for_acrt_thread_detach 000000018000510c f   MSVCRT:ucrt_stubs.obj
 0001:0000410c       __scrt_stub_for_acrt_uninitialize 000000018000510c f   MSVCRT:ucrt_stubs.obj
 0001:0000410c       __scrt_stub_for_acrt_uninitialize_critical 000000018000510c f   MSVCRT:ucrt_stubs.obj
 0001:0000410c       __vcrt_initialize          000000018000510c f   MSVCRT:ucrt_stubs.obj
 0001:0000410c       __vcrt_thread_attach       000000018000510c f   MSVCRT:ucrt_stubs.obj
 0001:0000410c       __vcrt_thread_detach       000000018000510c f   MSVCRT:ucrt_stubs.obj
 0001:0000410c       __vcrt_uninitialize        000000018000510c f   MSVCRT:ucrt_stubs.obj
 0001:0000410c       __vcrt_uninitialize_critical 000000018000510c f   MSVCRT:ucrt_stubs.obj
 0001:00004110       __scrt_stub_for_is_c_termination_complete 0000000180005110 f   MSVCRT:ucrt_stubs.obj
 0001:00004110       _is_c_termination_complete 0000000180005110 f   MSVCRT:ucrt_stubs.obj
 0001:00004130       _guard_dispatch_icall_nop  0000000180005130 f   MSVCRT:guard_dispatch.obj
 0001:00004150       _guard_xfg_dispatch_icall_nop 0000000180005150 f   MSVCRT:guard_xfg_dispatch.obj
 0002:00000000       __imp_RtlCaptureContext    0000000180006000     kernel32:KERNEL32.dll
 0002:00000008       __imp_RtlLookupFunctionEntry 0000000180006008     kernel32:KERNEL32.dll
 0002:00000010       __imp_RtlVirtualUnwind     0000000180006010     kernel32:KERNEL32.dll
 0002:00000018       __imp_UnhandledExceptionFilter 0000000180006018     kernel32:KERNEL32.dll
 0002:00000020       __imp_SetUnhandledExceptionFilter 0000000180006020     kernel32:KERNEL32.dll
 0002:00000028       __imp_GetCurrentProcess    0000000180006028     kernel32:KERNEL32.dll
 0002:00000030       __imp_TerminateProcess     0000000180006030     kernel32:KERNEL32.dll
 0002:00000038       __imp_IsProcessorFeaturePresent 0000000180006038     kernel32:KERNEL32.dll
 0002:00000040       __imp_CloseHandle          0000000180006040     kernel32:KERNEL32.dll
 0002:00000048       __imp_InitializeCriticalSectionAndSpinCount 0000000180006048     kernel32:KERNEL32.dll
 0002:00000050       __imp_DeleteCriticalSection 0000000180006050     kernel32:KERNEL32.dll
 0002:00000058       __imp_CreateEventW         0000000180006058     kernel32:KERNEL32.dll
 0002:00000060       __imp_GetModuleHandleW     0000000180006060     kernel32:KERNEL32.dll
 0002:00000068       __imp_GetProcAddress       0000000180006068     kernel32:KERNEL32.dll
 0002:00000070       __imp_IsDebuggerPresent    0000000180006070     kernel32:KERNEL32.dll
 0002:00000078       __imp_QueryPerformanceCounter 0000000180006078     kernel32:KERNEL32.dll
 0002:00000080       __imp_GetCurrentProcessId  0000000180006080     kernel32:KERNEL32.dll
 0002:00000088       __imp_GetCurrentThreadId   0000000180006088     kernel32:KERNEL32.dll
 0002:00000090       __imp_GetSystemTimeAsFileTime 0000000180006090     kernel32:KERNEL32.dll
 0002:00000098       __imp_DisableThreadLibraryCalls 0000000180006098     kernel32:KERNEL32.dll
 0002:000000a0       __imp_InitializeSListHead  00000001800060a0     kernel32:KERNEL32.dll
 0002:000000a8       \177KERNEL32_NULL_THUNK_DATA 00000001800060a8     kernel32:KERNEL32.dll
 0002:000000b0       __imp_memcpy               00000001800060b0     vcruntime:VCRUNTIME140.dll
 0002:000000b8       __imp_memset               00000001800060b8     vcruntime:VCRUNTIME140.dll
 0002:000000c0       __imp_strchr               00000001800060c0     vcruntime:VCRUNTIME140.dll
 0002:000000c8       __imp___C_specific_handler 00000001800060c8     vcruntime:VCRUNTIME140.dll
 0002:000000d0       __imp___std_type_info_destroy_list 00000001800060d0     vcruntime:VCRUNTIME140.dll
 0002:000000d8       \177VCRUNTIME140_NULL_THUNK_DATA 00000001800060d8     vcruntime:VCRUNTIME140.dll
 0002:000000e0       __imp_malloc               00000001800060e0     ucrt:api-ms-win-crt-heap-l1-1-0.dll
 0002:000000e8       __imp_free                 00000001800060e8     ucrt:api-ms-win-crt-heap-l1-1-0.dll
 0002:000000f0       \177api-ms-win-crt-heap-l1-1-0_NULL_THUNK_DATA 00000001800060f0     ucrt:api-ms-win-crt-heap-l1-1-0.dll
 0002:000000f8       __imp__errno               00000001800060f8     ucrt:api-ms-win-crt-runtime-l1-1-0.dll
 0002:00000100       __imp_exit                 0000000180006100     ucrt:api-ms-win-crt-runtime-l1-1-0.dll
 0002:00000108       __imp__cexit               0000000180006108     ucrt:api-ms-win-crt-runtime-l1-1-0.dll
 0002:00000110       __imp__crt_atexit          0000000180006110     ucrt:api-ms-win-crt-runtime-l1-1-0.dll
 0002:00000118       __imp__execute_onexit_table 0000000180006118     ucrt:api-ms-win-crt-runtime-l1-1-0.dll
 0002:00000120       __imp__register_onexit_function 0000000180006120     ucrt:api-ms-win-crt-runtime-l1-1-0.dll
 0002:00000128       __imp__initialize_onexit_table 0000000180006128     ucrt:api-ms-win-crt-runtime-l1-1-0.dll
 0002:00000130       __imp__initialize_narrow_environment 0000000180006130     ucrt:api-ms-win-crt-runtime-l1-1-0.dll
 0002:00000138       __imp__configure_narrow_argv 0000000180006138     ucrt:api-ms-win-crt-runtime-l1-1-0.dll
 0002:00000140       __imp__seh_filter_dll      0000000180006140     ucrt:api-ms-win-crt-runtime-l1-1-0.dll
 0002:00000148       __imp__initterm_e          0000000180006148     ucrt:api-ms-win-crt-runtime-l1-1-0.dll
 0002:00000150       __imp__initterm            0000000180006150     ucrt:api-ms-win-crt-runtime-l1-1-0.dll
 0002:00000158       \177api-ms-win-crt-runtime-l1-1-0_NULL_THUNK_DATA 0000000180006158     ucrt:api-ms-win-crt-runtime-l1-1-0.dll
 0002:00000160       __imp___acrt_iob_func      0000000180006160     ucrt:api-ms-win-crt-stdio-l1-1-0.dll
 0002:00000168       __imp_fflush               0000000180006168     ucrt:api-ms-win-crt-stdio-l1-1-0.dll
 0002:00000170       __imp___stdio_common_vsprintf 0000000180006170     ucrt:api-ms-win-crt-stdio-l1-1-0.dll
 0002:00000178       __imp___stdio_common_vfprintf 0000000180006178     ucrt:api-ms-win-crt-stdio-l1-1-0.dll
 0002:00000180       \177api-ms-win-crt-stdio-l1-1-0_NULL_THUNK_DATA 0000000180006180     ucrt:api-ms-win-crt-stdio-l1-1-0.dll
 0002:00000188       __imp_strcmp               0000000180006188     ucrt:api-ms-win-crt-string-l1-1-0.dll
 0002:00000190       __imp_strcpy               0000000180006190     ucrt:api-ms-win-crt-string-l1-1-0.dll
 0002:00000198       __imp__strdup              0000000180006198     ucrt:api-ms-win-crt-string-l1-1-0.dll
 0002:00000198       __imp_strdup               0000000180006198     ucrt:api-ms-win-crt-string-l1-1-0.dll
 0002:000001a0       __imp_strlen               00000001800061a0     ucrt:api-ms-win-crt-string-l1-1-0.dll
 0002:000001a8       __imp_strncpy              00000001800061a8     ucrt:api-ms-win-crt-string-l1-1-0.dll
 0002:000001b0       \177api-ms-win-crt-string-l1-1-0_NULL_THUNK_DATA 00000001800061b0     ucrt:api-ms-win-crt-string-l1-1-0.dll
 0002:000001b8       __guard_check_icall_fptr   00000001800061b8     MSVCRT:guard_support.obj
 0002:000001c0       __guard_xfg_check_icall_fptr 00000001800061c0     MSVCRT:guard_support.obj
 0002:000001c8       __guard_dispatch_icall_fptr 00000001800061c8     MSVCRT:guard_support.obj
 0002:000001d0       __guard_xfg_dispatch_icall_fptr 00000001800061d0     MSVCRT:guard_support.obj
 0002:000001d8       __guard_xfg_table_dispatch_icall_fptr 00000001800061d8     MSVCRT:guard_support.obj
 0002:000001e0       __castguard_check_failure_os_handled_fptr 00000001800061e0     MSVCRT:guard_support.obj
 0002:000001e8       __guard_memcpy_fptr        00000001800061e8     vcruntime:softmemtag.obj
 0002:000001f0       __xc_a                     00000001800061f0     MSVCRT:initializers.obj
 0002:000001f8       __xc_z                     00000001800061f8     MSVCRT:initializers.obj
 0002:00000200       __xi_a                     0000000180006200     MSVCRT:initializers.obj
 0002:00000210       __xi_z                     0000000180006210     MSVCRT:initializers.obj
 0002:00000218       __xl_a                     0000000180006218     MSVCRT:tlssup.obj
 0002:00000220       __xl_z                     0000000180006220     MSVCRT:tlssup.obj
 0002:00000228       __xp_a                     0000000180006228     MSVCRT:initializers.obj
 0002:00000230       __xp_z                     0000000180006230     MSVCRT:initializers.obj
 0002:00000238       __xt_a                     0000000180006238     MSVCRT:initializers.obj
 0002:00000240       __xt_z                     0000000180006240     MSVCRT:initializers.obj
 0002:00000250       ??_C@_0BG@IKDDPPGD@?$CILjava?1lang?1String?$DL?$CJV@ 0000000180006250     libattach039Agent00.obj
 0002:00000270       g_refKindStr               0000000180006270     libattach039Agent00.obj
 0002:00000420       ??_C@_09BPLDFGCI@unknown_0@ 0000000180006420     libattach039Agent00.obj
 0002:00000430       ??_C@_0BL@FPNMECJD@JVMTI_HEAP_REFERENCE_CLASS@ 0000000180006430     libattach039Agent00.obj
 0002:00000450       ??_C@_0BL@FKGKKLNM@JVMTI_HEAP_REFERENCE_FIELD@ 0000000180006450     libattach039Agent00.obj
 0002:00000470       ??_C@_0CD@CAEHCFJF@JVMTI_HEAP_REFERENCE_ARRAY_ELEM@ 0000000180006470     libattach039Agent00.obj
 0002:00000498       ??_C@_0CC@DNEBMCNK@JVMTI_HEAP_REFERENCE_CLASS_LOAD@ 0000000180006498     libattach039Agent00.obj
 0002:000004c0       ??_C@_0BN@CJMIPEBB@JVMTI_HEAP_REFERENCE_SIGNERS@ 00000001800064c0     libattach039Agent00.obj
 0002:000004e0       ??_C@_0CH@HBOIDPEB@JVMTI_HEAP_REFERENCE_PROTECTION@ 00000001800064e0     libattach039Agent00.obj
 0002:00000508       ??_C@_0BP@MDKGDGKL@JVMTI_HEAP_REFERENCE_INTERFACE@ 0000000180006508     libattach039Agent00.obj
 0002:00000528       ??_C@_0CC@JJMIHNJH@JVMTI_HEAP_REFERENCE_STATIC_FIE@ 0000000180006528     libattach039Agent00.obj
 0002:00000550       ??_C@_0CD@IDHEEGID@JVMTI_HEAP_REFERENCE_CONSTANT_P@ 0000000180006550     libattach039Agent00.obj
 0002:00000578       ??_C@_0CA@EFFCHNG@JVMTI_HEAP_REFERENCE_SUPERCLASS@ 0000000180006578     libattach039Agent00.obj
 0002:00000598       ??_C@_0L@PCDFHGCJ@unknown_11@ 0000000180006598     libattach039Agent00.obj
 0002:000005a8       ??_C@_0L@NJBICFOK@unknown_12@ 00000001800065a8     libattach039Agent00.obj
 0002:000005b8       ??_C@_0L@MAADBEKL@unknown_13@ 00000001800065b8     libattach039Agent00.obj
 0002:000005c8       ??_C@_0L@IPECICGM@unknown_14@ 00000001800065c8     libattach039Agent00.obj
 0002:000005d8       ??_C@_0L@JGFJLDCN@unknown_15@ 00000001800065d8     libattach039Agent00.obj
 0002:000005e8       ??_C@_0L@LNHEOAOO@unknown_16@ 00000001800065e8     libattach039Agent00.obj
 0002:000005f8       ??_C@_0L@KEGPNBKP@unknown_17@ 00000001800065f8     libattach039Agent00.obj
 0002:00000608       ??_C@_0L@CDPHMNGA@unknown_18@ 0000000180006608     libattach039Agent00.obj
 0002:00000618       ??_C@_0L@DKOMPMCB@unknown_19@ 0000000180006618     libattach039Agent00.obj
 0002:00000628       ??_C@_0L@OJGIPJDB@unknown_20@ 0000000180006628     libattach039Agent00.obj
 0002:00000638       ??_C@_0CA@KAOFNDEM@JVMTI_HEAP_REFERENCE_JNI_GLOBAL@ 0000000180006638     libattach039Agent00.obj
 0002:00000658       ??_C@_0CC@HPFAJBK@JVMTI_HEAP_REFERENCE_SYSTEM_CLA@ 0000000180006658     libattach039Agent00.obj
 0002:00000680       ??_C@_0BN@FDEGFOHC@JVMTI_HEAP_REFERENCE_MONITOR@ 0000000180006680     libattach039Agent00.obj
 0002:000006a0       ??_C@_0CB@HKIBCMAJ@JVMTI_HEAP_REFERENCE_STACK_LOCA@ 00000001800066a0     libattach039Agent00.obj
 0002:000006c8       ??_C@_0BP@EAACMMOE@JVMTI_HEAP_REFERENCE_JNI_LOCAL@ 00000001800066c8     libattach039Agent00.obj
 0002:000006e8       ??_C@_0BM@IJDEOGOE@JVMTI_HEAP_REFERENCE_THREAD@ 00000001800066e8     libattach039Agent00.obj
 0002:00000708       ??_C@_0BL@EDGPPKC@JVMTI_HEAP_REFERENCE_OTHER@ 0000000180006708     libattach039Agent00.obj
 0002:00000724       ??_C@_04BCJPDBDA@Code@     0000000180006724     libattach039Agent00.obj
 0002:00000730       ??_C@_0BA@OCLMCFKC@LineNumberTable@ 0000000180006730     libattach039Agent00.obj
 0002:00000740       ??_C@_0BD@CPAEPILC@LocalVariableTable@ 0000000180006740     libattach039Agent00.obj
 0002:00000758       ??_C@_0BH@NMBDNHBD@LocalVariableTypeTable@ 0000000180006758     libattach039Agent00.obj
 0002:00000770       ??_C@_0O@HIHEEDNJ@StackMapTable@ 0000000180006770     libattach039Agent00.obj
 0002:00000780       ??_C@_0CN@NKCKIIJI@nsk?1share?1aod?1TargetApplication@ 0000000180006780     libattach039Agent00.obj
 0002:000007b0       ??_C@_0M@OANFKLGH@agentLoaded@ 00000001800067b0     libattach039Agent00.obj
 0002:000007c0       ??_C@_0O@JINEPNAJ@agentFinished@ 00000001800067c0     libattach039Agent00.obj
 0002:000007d0       ??_C@_0BH@BOPHNJNA@?$CILjava?1lang?1String?$DLZ?$CJV@ 00000001800067d0     libattach039Agent00.obj
 0002:000007e8       ??_C@_0L@HCDIAMJG@?9?5?$CFs?0?5?$CFd?3?5@ 00000001800067e8     libattach039Agent00.obj
 0002:00000800       ??_C@_0JI@HLPECLFI@?$CD?5?4?4?4?6?$CD?5ERROR?3?5too?5many?5complai@ 0000000180006800     libattach039Agent00.obj
 0002:000008a0       ??_C@_0ED@JNEKCCOB@The?5following?5fake?5exception?5st@ 00000001800068a0     libattach039Agent00.obj
 0002:000008e8       ??_C@_0CN@FCNMDFBH@nsk?4share?4Fake_Exception_for_RU@ 00000001800068e8     libattach039Agent00.obj
 0002:00000918       ??_C@_08PGFFNAEI@?$CI?$CFs?3?$CFd?$CJ?5@ 0000000180006918     libattach039Agent00.obj
 0002:00000928       ??_C@_0DP@IENMAEGI@s?2test?2hotspot?2jtreg?2vmTestbase@ 0000000180006928     libattach039Agent00.obj
 0002:00000968       ??_C@_0BL@NDJLFFJB@?7at?5nsk_lvcomplain?$CI?$CFs?3?$CFd?$CJ?6@ 0000000180006968     libattach039Agent00.obj
 0002:00000988       ??_C@_0BC@JOOKAFKF@?$CD?5ERROR?3?5?$CFs?0?5?$CFd?3?5@ 0000000180006988     libattach039Agent00.obj
 0002:000009a0       ??_C@_09KJEAHMEH@?$CD?5ERROR?3?5@ 00000001800069a0     libattach039Agent00.obj
 0002:000009ac       ??_C@_02GPIOPFAK@?$DO?$DO@ 00000001800069ac     libattach039Agent00.obj
 0002:000009b0       ??_C@_02FODMEDOG@?$DM?$DM@ 00000001800069b0     libattach039Agent00.obj
 0002:000009b4       ??_C@_02DJGKEECL@?4?4@     00000001800069b4     libattach039Agent00.obj
 0002:000009b8       ??_C@_0O@CJPGJOAF@?9?5?$CFs?0?5?$CFd?3?5?$CFs?5@ 00000001800069b8     libattach039Agent00.obj
 0002:000009c8       ??_C@_0CB@IAKPDOIC@?$CD?5?5?5verified?5assertion?5is?5FALSE@ 00000001800069c8     libattach039Agent00.obj
 0002:000009f0       ??_C@_0CO@LGONDEPD@stdout?3?5fflush?5failed?5?9?5err?$DN?$CFd?5@ 00000001800069f0     libattach039Agent00.obj
 0002:00000a20       ??_C@_0CO@KBGKJPBD@stderr?3?5fflush?5failed?5?9?5err?$DN?$CFd?5@ 0000000180006a20     libattach039Agent00.obj
 0002:00000a50       ??_C@_0BB@JCNMKLLK@JVMTI_ERROR_NONE@ 0000000180006a50     libattach039Agent00.obj
 0002:00000a68       ??_C@_0BL@LDIMKLPH@JVMTI_ERROR_INVALID_THREAD@ 0000000180006a68     libattach039Agent00.obj
 0002:00000a88       ??_C@_0CB@PJFPAIKJ@JVMTI_ERROR_INVALID_THREAD_GROU@ 0000000180006a88     libattach039Agent00.obj
 0002:00000ab0       ??_C@_0BN@LLMKHMNF@JVMTI_ERROR_INVALID_PRIORITY@ 0000000180006ab0     libattach039Agent00.obj
 0002:00000ad0       ??_C@_0CB@MBOFKAGB@JVMTI_ERROR_THREAD_NOT_SUSPENDE@ 0000000180006ad0     libattach039Agent00.obj
 0002:00000af8       ??_C@_0BN@FABOLPBI@JVMTI_ERROR_THREAD_SUSPENDED@ 0000000180006af8     libattach039Agent00.obj
 0002:00000b18       ??_C@_0BN@FDGNOBJM@JVMTI_ERROR_THREAD_NOT_ALIVE@ 0000000180006b18     libattach039Agent00.obj
 0002:00000b38       ??_C@_0BL@GOBIFKNJ@JVMTI_ERROR_INVALID_OBJECT@ 0000000180006b38     libattach039Agent00.obj
 0002:00000b58       ??_C@_0BK@FCMAJPPC@JVMTI_ERROR_INVALID_CLASS@ 0000000180006b58     libattach039Agent00.obj
 0002:00000b78       ??_C@_0BP@IKLLBKEB@JVMTI_ERROR_CLASS_NOT_PREPARED@ 0000000180006b78     libattach039Agent00.obj
 0002:00000b98       ??_C@_0BN@KLPPLKG@JVMTI_ERROR_INVALID_METHODID@ 0000000180006b98     libattach039Agent00.obj
 0002:00000bb8       ??_C@_0BN@BCEKOKND@JVMTI_ERROR_INVALID_LOCATION@ 0000000180006bb8     libattach039Agent00.obj
 0002:00000bd8       ??_C@_0BM@DFDGPME@JVMTI_ERROR_INVALID_FIELDID@ 0000000180006bd8     libattach039Agent00.obj
 0002:00000bf8       ??_C@_0BL@NELIEPEC@JVMTI_ERROR_NO_MORE_FRAMES@ 0000000180006bf8     libattach039Agent00.obj
 0002:00000c18       ??_C@_0BJ@BDBECFDM@JVMTI_ERROR_OPAQUE_FRAME@ 0000000180006c18     libattach039Agent00.obj
 0002:00000c38       ??_C@_0BK@MIIFNLOB@JVMTI_ERROR_TYPE_MISMATCH@ 0000000180006c38     libattach039Agent00.obj
 0002:00000c58       ??_C@_0BJ@HPCAOILC@JVMTI_ERROR_INVALID_SLOT@ 0000000180006c58     libattach039Agent00.obj
 0002:00000c78       ??_C@_0BG@CHILOPNI@JVMTI_ERROR_DUPLICATE@ 0000000180006c78     libattach039Agent00.obj
 0002:00000c90       ??_C@_0BG@DIEMLHKM@JVMTI_ERROR_NOT_FOUND@ 0000000180006c90     libattach039Agent00.obj
 0002:00000ca8       ??_C@_0BM@NHMCKHOB@JVMTI_ERROR_INVALID_MONITOR@ 0000000180006ca8     libattach039Agent00.obj
 0002:00000cc8       ??_C@_0BO@PPEDAJGL@JVMTI_ERROR_NOT_MONITOR_OWNER@ 0000000180006cc8     libattach039Agent00.obj
 0002:00000ce8       ??_C@_0BG@FCAIPEID@JVMTI_ERROR_INTERRUPT@ 0000000180006ce8     libattach039Agent00.obj
 0002:00000d00       ??_C@_0CB@EGDBNKOI@JVMTI_ERROR_INVALID_CLASS_FORMA@ 0000000180006d00     libattach039Agent00.obj
 0002:00000d28       ??_C@_0CG@DGKOGIAL@JVMTI_ERROR_CIRCULAR_CLASS_DEFI@ 0000000180006d28     libattach039Agent00.obj
 0002:00000d50       ??_C@_0BP@ICEALPKC@JVMTI_ERROR_FAILS_VERIFICATION@ 0000000180006d50     libattach039Agent00.obj
 0002:00000d70       ??_C@_0DC@JDACLMIO@JVMTI_ERROR_UNSUPPORTED_REDEFIN@ 0000000180006d70     libattach039Agent00.obj
 0002:00000da8       ??_C@_0DE@GKDKNOMJ@JVMTI_ERROR_UNSUPPORTED_REDEFIN@ 0000000180006da8     libattach039Agent00.obj
 0002:00000de0       ??_C@_0BO@LAFKIOG@JVMTI_ERROR_INVALID_TYPESTATE@ 0000000180006de0     libattach039Agent00.obj
 0002:00000e00       ??_C@_0DH@INDGCLLB@JVMTI_ERROR_UNSUPPORTED_REDEFIN@ 0000000180006e00     libattach039Agent00.obj
 0002:00000e38       ??_C@_0DE@NHEOMMGI@JVMTI_ERROR_UNSUPPORTED_REDEFIN@ 0000000180006e38     libattach039Agent00.obj
 0002:00000e70       ??_C@_0CA@EKPNJOEP@JVMTI_ERROR_UNSUPPORTED_VERSION@ 0000000180006e70     libattach039Agent00.obj
 0002:00000e90       ??_C@_0BN@OFFMAHHL@JVMTI_ERROR_NAMES_DONT_MATCH@ 0000000180006e90     libattach039Agent00.obj
 0002:00000eb0       ??_C@_0DN@HHBBLAKE@JVMTI_ERROR_UNSUPPORTED_REDEFIN@ 0000000180006eb0     libattach039Agent00.obj
 0002:00000ef0       ??_C@_0DO@HMBGBGNA@JVMTI_ERROR_UNSUPPORTED_REDEFIN@ 0000000180006ef0     libattach039Agent00.obj
 0002:00000f30       ??_C@_0BP@PBECGKHJ@JVMTI_ERROR_UNMODIFIABLE_CLASS@ 0000000180006f30     libattach039Agent00.obj
 0002:00000f50       ??_C@_0BK@CANILEHF@JVMTI_ERROR_NOT_AVAILABLE@ 0000000180006f50     libattach039Agent00.obj
 0002:00000f70       ??_C@_0CE@INJKMEFK@JVMTI_ERROR_MUST_POSSESS_CAPABI@ 0000000180006f70     libattach039Agent00.obj
 0002:00000f98       ??_C@_0BJ@LBFPFPDM@JVMTI_ERROR_NULL_POINTER@ 0000000180006f98     libattach039Agent00.obj
 0002:00000fb8       ??_C@_0BP@CHJPNNEM@JVMTI_ERROR_ABSENT_INFORMATION@ 0000000180006fb8     libattach039Agent00.obj
 0002:00000fd8       ??_C@_0BP@OMFMNLC@JVMTI_ERROR_INVALID_EVENT_TYPE@ 0000000180006fd8     libattach039Agent00.obj
 0002:00000ff8       ??_C@_0BN@BIBNPHHO@JVMTI_ERROR_ILLEGAL_ARGUMENT@ 0000000180006ff8     libattach039Agent00.obj
 0002:00001018       ??_C@_0BK@KKNDHDCE@JVMTI_ERROR_NATIVE_METHOD@ 0000000180007018     libattach039Agent00.obj
 0002:00001038       ??_C@_0BK@PMKCFHAE@JVMTI_ERROR_OUT_OF_MEMORY@ 0000000180007038     libattach039Agent00.obj
 0002:00001058       ??_C@_0BK@NNJBDMNB@JVMTI_ERROR_ACCESS_DENIED@ 0000000180007058     libattach039Agent00.obj
 0002:00001078       ??_C@_0BI@GHECLMNC@JVMTI_ERROR_WRONG_PHASE@ 0000000180007078     libattach039Agent00.obj
 0002:00001090       ??_C@_0BF@OLIHJOII@JVMTI_ERROR_INTERNAL@ 0000000180007090     libattach039Agent00.obj
 0002:000010a8       ??_C@_0BO@EOHGKJHI@JVMTI_ERROR_UNATTACHED_THREAD@ 00000001800070a8     libattach039Agent00.obj
 0002:000010c8       ??_C@_0CA@LKHFDACL@JVMTI_ERROR_INVALID_ENVIRONMENT@ 00000001800070c8     libattach039Agent00.obj
 0002:000010e8       ??_C@_0BA@MMFHLOKK@?$DMunknown?5error?$DO@ 00000001800070e8     libattach039Agent00.obj
 0002:000010f8       ??_C@_0CF@CBHOKDB@throwable?5?$DN?5jni?9?$DOExceptionOccur@ 00000001800070f8     libattach039Agent00.obj
 0002:00001120       ??_C@_03OFAPEBGM@?$CFs?6@  0000000180007120     libattach039Agent00.obj
 0002:00001128       ??_C@_0DM@LPIGEGNJ@s?2test?2hotspot?2jtreg?2vmTestbase@ 0000000180007128     libattach039Agent00.obj
 0002:00001168       ??_C@_0CC@NFCNPEPK@Exception?5in?5JNI?5call?5?$CIcleared?$CJ@ 0000000180007168     libattach039Agent00.obj
 0002:00001190       ??_C@_0BJ@IBAKFIKF@jni?9?$DOExceptionDescribe?$CI?$CJ@ 0000000180007190     libattach039Agent00.obj
 0002:000011b0       ??_C@_0BG@GGKALKMH@jni?9?$DOExceptionClear?$CI?$CJ@ 00000001800071b0     libattach039Agent00.obj
 0002:000011c8       ??_C@_0CF@JMGFGJLJ@?$CD?5?5?5verified?5JNI?5assertion?5is?5F@ 00000001800071c8     libattach039Agent00.obj
 0002:000011f0       ??_C@_0CB@MLNJNCLJ@?5?5jvmti?5error?3?5code?$DN?$CFd?0?5name?$DN?$CFs@ 00000001800071f0     libattach039Agent00.obj
 0002:00001218       ??_C@_0CD@OHBGDKMK@?$CD?5?5?5jvmti?5error?3?5code?$DN?$CFd?0?5name?$DN@ 0000000180007218     libattach039Agent00.obj
 0002:00001240       ??_C@_0CG@JNNCGPHB@?$CD?5?5?5error?5expected?3?5code?$DN?$CFd?0?5na@ 0000000180007240     libattach039Agent00.obj
 0002:00001270       ??_C@_0EB@IMGKPCGE@?$CIstr_obj?5?$DN?5jni?9?$DONewStringUTF?$CIco@ 0000000180007270     libattach039Agent00.obj
 0002:000012c0       ??_C@_0EA@HFOGGBCC@s?2test?2hotspot?2jtreg?2vmTestbase@ 00000001800072c0     libattach039Agent00.obj
 0002:00001300       ??_C@_05KKCIMGE@error@     0000000180007300     libattach039Agent00.obj
 0002:00001308       ??_C@_0CJ@JACLEAA@Test?5failed?5by?5setFailStatus?$CI?$CJ?4@ 0000000180007308     libattach039Agent00.obj
 0002:00001338       ??_C@_0BD@HGNAOMCP@agent_data_monitor@ 0000000180007338     libattach039Agent00.obj
 0002:00001350       ??_C@_0EB@OGCLGKLN@javaVM?9?$DOGetEnv?$CI?$CIvoid?5?$CK?$CK?$CJ?$CGjvmti_@ 0000000180007350     libattach039Agent00.obj
 0002:000013a0       ??_C@_0EA@PNBCDMOA@s?2test?2hotspot?2jtreg?2vmTestbase@ 00000001800073a0     libattach039Agent00.obj
 0002:000013e0       ??_C@_0CI@DDPIFBGM@init_agent_data?$CIjvmti_env?0?5?$CGage@ 00000001800073e0     libattach039Agent00.obj
 0002:00001408       ??_C@_0DI@ILAHDLMP@?$CI?$CKagentThreadProc?$CJ?$CIjvmti_env?0?5a@ 0000000180007408     libattach039Agent00.obj
 0002:00001440       ??_C@_0BD@KDBALNLB@JVMTI?5agent?5thread@ 0000000180007440     libattach039Agent00.obj
 0002:00001458       ??_C@_0BB@NOKBFPFO@java?1lang?1Thread@ 0000000180007458     libattach039Agent00.obj
 0002:0000146c       ??_C@_06FALKBLGB@?$DMinit?$DO@ 000000018000746c     libattach039Agent00.obj
 0002:00001480       ??_C@_0EB@IFJBFEKC@?$CIthreadClass?5?$DN?5jni_env?9?$DOFindCla@ 0000000180007480     libattach039Agent00.obj
 0002:000014d0       ??_C@_0GF@FGFIBKKL@?$CIthreadCtor?5?$DN?5jni_env?9?$DOGetMetho@ 00000001800074d0     libattach039Agent00.obj
 0002:00001538       ??_C@_0DN@NCPDJLOG@?$CIthreadName?5?$DN?5jni_env?9?$DONewStrin@ 0000000180007538     libattach039Agent00.obj
 0002:00001580       ??_C@_0FE@PFKODBGC@?$CIthreadObject?5?$DN?5jni_env?9?$DONewObj@ 0000000180007580     libattach039Agent00.obj
 0002:000015e0       ??_C@_0ED@HOBAHHJI@?$CIthreadGlobalRef?5?$DN?5jni_env?9?$DONew@ 00000001800075e0     libattach039Agent00.obj
 0002:00001630       ??_C@_0FN@HNJJAHFC@jvmti_env?9?$DORunAgentThread?$CIagent@ 0000000180007630     libattach039Agent00.obj
 0002:00001690       ??_C@_0EA@MOJDNKDF@Debuggee?5status?5sync?5aborted?5be@ 0000000180007690     libattach039Agent00.obj
 0002:000016d0       ??_C@_0EA@EEOEJAEN@status?5?$DN?5syncDebuggeeStatus?$CIjni@ 00000001800076d0     libattach039Agent00.obj
 0002:00001710       ??_C@_0BL@JBCFNBMB@nsk_jvmti_resetAgentData?$CI?$CJ@ 0000000180007710     libattach039Agent00.obj
 0002:00001730       ??_C@_0EL@LPBEELIP@s?2test?2hotspot?2jtreg?2vmTestbase@ 0000000180007730     libattach039Agent00.obj
 0002:00001780       ??_C@_0CK@JDAMFDMJ@jvmti?9?$DOSetTag?$CIo?0?5tag?$CJ?5?$DN?$DN?5JVMTI_@ 0000000180007780     libattach039Agent00.obj
 0002:000017b0       ??_C@_0CC@DAMNHKNI@Can?8t?5set?5tag?5?$CFli?5for?5object?5?$CFl@ 00000001800077b0     libattach039Agent00.obj
 0002:000017d8       ??_C@_0DL@HAJPNKEF@jvmti?9?$DOGetObjectHashCode?$CIo?0?5?$CGha@ 00000001800077d8     libattach039Agent00.obj
 0002:00001818       ??_C@_0BL@JFPIEOBF@Can?8t?5get?5hash?5object?5?$CFlx?6@ 0000000180007818     libattach039Agent00.obj
 0002:00001838       ??_C@_0BG@DICPHBKN@setTag?3?5?$CF08x?5?$DM?9?5?$CF?53li@ 0000000180007838     libattach039Agent00.obj
 0002:00001850       ??_C@_0DH@FCEEBDMJ@?$CIs?5?$DN?5jni?9?$DOGetStringUTFChars?$CIsIn@ 0000000180007850     libattach039Agent00.obj
 0002:00001888       ??_C@_0BJ@OKKGHDCN@Can?8t?5get?5string?5at?5?$CF?$CDp?6@ 0000000180007888     libattach039Agent00.obj
 0002:000018a8       ??_C@_0BP@EKFLGGFJ@Can?8t?5get?5string?5at?5?$CF?$CDp?3?5null?6@ 00000001800078a8     libattach039Agent00.obj
 0002:000018c8       ??_C@_06ICODBHCL@?5?1?1?5?$CFs@ 00000001800078c8     libattach039Agent00.obj
 0002:000018d0       ??_C@_0DB@KGFPLEGO@?$CIr?5?$DN?5jvmti?9?$DOGetTag?$CIo?0?5?$CGtag?$CJ?$CJ?5?$DN?$DN@ 00000001800078d0     libattach039Agent00.obj
 0002:00001908       ??_C@_0CO@PDAGBCGJ@Can?8t?5GetTag?5for?5object?5?$CFlx?4?5Re@ 0000000180007908     libattach039Agent00.obj
 0002:00001938       ??_C@_0CH@HPEODOHC@TEST_BUG?3?5Max?4?5number?5of?5refs?5r@ 0000000180007938     libattach039Agent00.obj
 0002:00001960       ??_C@_0DI@PHFCABIM@?$CIr?5?$DN?5jvmti?9?$DOGetTag?$CIfrom?0?5?$CGtagFr@ 0000000180007960     libattach039Agent00.obj
 0002:00001998       ??_C@_0DI@MDEGFNKD@TEST_BUG?3?5Can?8t?5GetTag?5for?5obje@ 0000000180007998     libattach039Agent00.obj
 0002:000019d0       ??_C@_0DE@MLELJAHM@?$CIr?5?$DN?5jvmti?9?$DOGetTag?$CIto?0?5?$CGtagTo?$CJ?$CJ@ 00000001800079d0     libattach039Agent00.obj
 0002:00001a08       ??_C@_0CF@NBAMCKHO@Unexpected?5exception?5after?5JNI?5@ 0000000180007a08     libattach039Agent00.obj
 0002:00001a30       ??_C@_0DG@ECLJIGOO@s?2test?2hotspot?2jtreg?2vmTestbase@ 0000000180007a30     libattach039Agent00.obj
 0002:00001a70       ??_C@_0EK@CABJMPML@WARNING?3?5some?5error?5happened?5in@ 0000000180007a70     libattach039Agent00.obj
 0002:00001ac0       ??_C@_0CN@EDIMGGCE@options?5were?5not?5passed?5to?5the?5@ 0000000180007ac0     libattach039Agent00.obj
 0002:00001af0       ??_C@_0BO@HIBNDEOE@Invalid?5options?5format?3?5?8?$CFs?8?6@ 0000000180007af0     libattach039Agent00.obj
 0002:00001b10       ??_C@_0BG@BCGDCLLA@Option?5?8?$CFs?8?5is?5empty?6@ 0000000180007b10     libattach039Agent00.obj
 0002:00001b30       ??_C@_0EI@CFFDGDKG@WARNING?3?5not?5all?5options?5were?5p@ 0000000180007b30     libattach039Agent00.obj
 0002:00001b80       ??_C@_0EN@LHKBBCDP@?$CIoptions?5?$DN?5?$CIOptions?$CK?$CJ?5nsk_aod_c@ 0000000180007b80     libattach039Agent00.obj
 0002:00001bd0       ??_C@_0DM@MFFOLIAC@nsk_aod_optionSpecified?$CIoptions@ 0000000180007bd0     libattach039Agent00.obj
 0002:00001c10       ??_C@_0L@DALKGIIP@?9agentName@ 0000000180007c10     libattach039Agent00.obj
 0002:00001c20       ??_C@_0BN@PFMBIOBG@Agent?5name?5wasn?8t?5specified?6@ 0000000180007c20     libattach039Agent00.obj
 0002:00001c40       ??_C@_08FBJJFDKJ@?9verbose@ 0000000180007c40     libattach039Agent00.obj
 0002:00001c4c       ??_C@_05LAPONLG@false@     0000000180007c4c     libattach039Agent00.obj
 0002:00001c58       ??_C@_0BD@FMBAOLJK@options?5?$CB?$DN?5nullptr@ 0000000180007c58     libattach039Agent00.obj
 0002:00001c70       ??_C@_0O@BPHJJCEJ@Options?5null?6@ 0000000180007c70     libattach039Agent00.obj
 0002:00001c80       ??_C@_0BL@NJPPLGIO@Option?5?8?$CFs?8?5isn?8t?5defined?6@ 0000000180007c80     libattach039Agent00.obj
 0002:00001ca0       ??_C@_0BE@DNNCOIDF@Agent?5?$CFs?5is?5loaded?6@ 0000000180007ca0     libattach039Agent00.obj
 0002:00001cc0       ??_C@_0EJ@NDOPGKMK@?$CIlocalTargetAppClass?5?$DN?5jni?9?$DOFin@ 0000000180007cc0     libattach039Agent00.obj
 0002:00001d10       ??_C@_0EO@HKMHFBAF@?$CItargetAppClass?5?$DN?5?$CIjclass?$CJ?5jni?9@ 0000000180007d10     libattach039Agent00.obj
 0002:00001d60       ??_C@_0IB@FFOAAHNN@?$CIagentLoadedMethod?5?$DN?5jni?9?$DOGetSt@ 0000000180007d60     libattach039Agent00.obj
 0002:00001de8       ??_C@_0DM@HLLJGLFL@?$CIagentNameString?5?$DN?5jni?9?$DONewStri@ 0000000180007de8     libattach039Agent00.obj
 0002:00001e30       ??_C@_0FP@EEAOJLDE@?$CFs?3?5TEST?5LOGIC?5ERROR?3?5method?5?8a@ 0000000180007e30     libattach039Agent00.obj
 0002:00001e90       ??_C@_0II@KPBFKHFM@Status?5of?5agent?5?8?$CFs?8?5is?5?8passed@ 0000000180007e90     libattach039Agent00.obj
 0002:00001f18       ??_C@_0CB@ECJEOOED@Agent?5?$CFs?5finished?5?$CIsuccess?3?5?$CFd?$CJ@ 0000000180007f18     libattach039Agent00.obj
 0002:00001f40       ??_C@_0IH@FIFEINGM@?$CIagentFinishedMethod?5?$DN?5jni?9?$DOGet@ 0000000180007f40     libattach039Agent00.obj
 0002:00001fc8       ??_C@_0P@POOJKNDK@jni?5?$CB?$DN?5nullptr@ 0000000180007fc8     libattach039Agent00.obj
 0002:00001fe0       ??_C@_0EC@LNOIGMCL@s?2test?2hotspot?2jtreg?2vmTestbase@ 0000000180007fe0     libattach039Agent00.obj
 0002:00002028       ??_C@_0BH@DFACKHAD@jvmti?9?$DODeallocate?$CImem?$CJ@ 0000000180008028     libattach039Agent00.obj
 0002:00002040       ??_C@_0BD@DPLLDHNC@Deallocate?5failed?6@ 0000000180008040     libattach039Agent00.obj
 0002:00002058       ??_C@_0CE@LGKCCDOO@jvmti?9?$DOGetThreadInfo?$CIthread?0?5?$CGi@ 0000000180008058     libattach039Agent00.obj
 0002:00002080       ??_C@_0BL@LNEBMKFE@Failed?5to?5get?5thread?5info?6@ 0000000180008080     libattach039Agent00.obj
 0002:000020a0       ??_C@_0ED@MGJECIFJ@jvmti?9?$DOSetEventNotificationMode@ 00000001800080a0     libattach039Agent00.obj
 0002:000020f0       ??_C@_0EC@OOBBODLO@jvmti?9?$DOSetEventNotificationMode@ 00000001800080f0     libattach039Agent00.obj
 0002:00002138       ??_C@_0DI@FCBOEPIP@?$CIklass?5?$DN?5jni?9?$DOFindClass?$CI?$CCjava?1l@ 0000000180008138     libattach039Agent00.obj
 0002:00002170       ??_C@_0CK@CNPMBPHM@Failed?5to?5get?5the?5java?4lang?4Thr@ 0000000180008170     libattach039Agent00.obj
 0002:000021a0       ??_C@_0CM@LKMKAAHP@Failed?5to?5get?5java?4lang?4Thread?5@ 00000001800081a0     libattach039Agent00.obj
 0002:000021d0       ??_C@_0CA@GPNPHECO@Failed?5to?5create?5Thread?5object?6@ 00000001800081d0     libattach039Agent00.obj
 0002:000021f0       ??_C@_0DA@LIFMFFL@?$CIthread?5?$DN?5jni?9?$DONewGlobalRef?$CIthr@ 00000001800081f0     libattach039Agent00.obj
 0002:00002220       ??_C@_0CD@DCJDOJMD@Failed?5to?5create?5global?5referen@ 0000000180008220     libattach039Agent00.obj
 0002:00002248       ??_C@_0DO@GADKBBKO@?$CIthreadNameString?5?$DN?5jni?9?$DONewStr@ 0000000180008248     libattach039Agent00.obj
 0002:00002290       ??_C@_0FM@BHODDBLA@?$CIthreadConstructor?5?$DN?5jni?9?$DOGetMe@ 0000000180008290     libattach039Agent00.obj
 0002:000022f0       ??_C@_0FB@LHHKAMDG@?$CIthread?5?$DN?5jni?9?$DONewObject?$CIklass?0@ 00000001800082f0     libattach039Agent00.obj
 0002:00002348       ??_C@_0DO@HGMCLGKA@?$CFs?3?5thread?5started?5from?5agent?5i@ 0000000180008348     libattach039Agent00.obj
 0002:00002390       ??_C@_0FI@JMNMBHCG@s?2test?2hotspot?2jtreg?2vmTestbase@ 0000000180008390     libattach039Agent00.obj
 0002:000023e8       ??_C@_0BF@EAJFPLBN@ThreadStartedByAgent@ 00000001800083e8     libattach039Agent00.obj
 0002:00002400       ??_C@_0BC@EOCLLCB@thread?5?$CB?$DN?5nullptr@ 0000000180008400     libattach039Agent00.obj
 0002:00002420       ??_C@_0FK@CHBJIDOM@jvmti?9?$DORunAgentThread?$CIthread?0?5s@ 0000000180008420     libattach039Agent00.obj
 0002:00002480       ??_C@_0BM@OKMFFMM@?$CFs?3?5new?5thread?5was?5started?6@ 0000000180008480     libattach039Agent00.obj
 0002:000024a0       ??_C@_0DC@GEMNJDJD@?$CFs?3?5ThreadEnd?5event?5was?5receive@ 00000001800084a0     libattach039Agent00.obj
 0002:000024d8       ??_C@_0CH@IPINKDLF@?$CFs?3?5ThreadStart?5event?5wasn?8t?5re@ 00000001800084d8     libattach039Agent00.obj
 0002:00002500       ??_C@_0CN@ECOHIHM@?$CFs?3?5started?5thread?5haven?8t?5exec@ 0000000180008500     libattach039Agent00.obj
 0002:00002530       ??_C@_0DE@KOBHNHPM@?$CFs?3?5ThreadStart?5event?5was?5recei@ 0000000180008530     libattach039Agent00.obj
 0002:00002568       ??_C@_0BB@CGPOECH@jvmti?5?$CB?$DN?5nullptr@ 0000000180008568     libattach039Agent00.obj
 0002:00002580       ??_C@_0EC@ODFGFOAJ@jvmti?9?$DOSetEventCallbacks?$CI?$CGevent@ 0000000180008580     libattach039Agent00.obj
 0002:000025c8       ??_C@_0BN@GGABIMJA@?$CFs?3?5initialization?5was?5done?6@ 00000001800085c8     libattach039Agent00.obj
 0002:000025e8       ??_C@_0CE@PACICCLF@nsk_aod_agentLoaded?$CIjni?0?5agentN@ 00000001800085e8     libattach039Agent00.obj
 0002:00002610       ??_C@_0BJ@CKPIAPN@?$CFs?3?5starting?5new?5thread?6@ 0000000180008610     libattach039Agent00.obj
 0002:00002630       ??_C@_0BL@GPCOJJBO@startNewThread?$CIjvmti?0?5jni?$CJ@ 0000000180008630     libattach039Agent00.obj
 0002:00002660       ??_C@_1EC@JIJBPKFM@?$AAa?$AAp?$AAi?$AA?9?$AAm?$AAs?$AA?9?$AAw?$AAi?$AAn?$AA?9?$AAc?$AAo?$AAr?$AAe@ 0000000180008660     MSVCRT:thread_safe_statics.obj
 0002:000026a8       ??_C@_1BK@MGMFAEKH@?$AAk?$AAe?$AAr?$AAn?$AAe?$AAl?$AA3?$AA2?$AA?4?$AAd?$AAl?$AAl@ 00000001800086a8     MSVCRT:thread_safe_statics.obj
 0002:000026c8       ??_C@_0BJ@JEBJOJFJ@SleepConditionVariableCS@ 00000001800086c8     MSVCRT:thread_safe_statics.obj
 0002:000026e8       ??_C@_0BJ@PGPPEPCC@WakeAllConditionVariable@ 00000001800086e8     MSVCRT:thread_safe_statics.obj
 0002:00002708       _pDefaultRawDllMain        0000000180008708     MSVCRT:dll_dllmain.obj
 0002:00002708       _pRawDllMain               0000000180008708     MSVCRT:dll_dllmain.obj
 0002:00002710       __xmm@ffffffffffffffffffffffffffffffff 0000000180008710     MSVCRT:utility.obj
 0002:00002720       _load_config_used          0000000180008720     MSVCRT:loadcfg.obj
 0002:00002900       _tls_used                  0000000180008900     MSVCRT:tlssup.obj
 0002:00002928       __volatile_metadata        0000000180008928     <linker-defined>
 0002:00002d08       __rtc_iaa                  0000000180008d08     MSVCRT:initsect.obj
 0002:00002d10       __rtc_izz                  0000000180008d10     MSVCRT:initsect.obj
 0002:00002d18       __rtc_taa                  0000000180008d18     MSVCRT:initsect.obj
 0002:00002d20       __rtc_tzz                  0000000180008d20     MSVCRT:initsect.obj
 0002:00002d28       _tls_start                 0000000180008d28     MSVCRT:tlssup.obj
 0002:00002d2c       _Init_thread_epoch         0000000180008d2c     MSVCRT:thread_safe_statics.obj
 0002:00002d30       _tls_end                   0000000180008d30     MSVCRT:tlssup.obj
 0002:00003484       __IMPORT_DESCRIPTOR_KERNEL32 0000000180009484     kernel32:KERNEL32.dll
 0002:00003498       __IMPORT_DESCRIPTOR_VCRUNTIME140 0000000180009498     vcruntime:VCRUNTIME140.dll
 0002:000034ac       __IMPORT_DESCRIPTOR_api-ms-win-crt-heap-l1-1-0 00000001800094ac     ucrt:api-ms-win-crt-heap-l1-1-0.dll
 0002:000034c0       __IMPORT_DESCRIPTOR_api-ms-win-crt-runtime-l1-1-0 00000001800094c0     ucrt:api-ms-win-crt-runtime-l1-1-0.dll
 0002:000034d4       __IMPORT_DESCRIPTOR_api-ms-win-crt-stdio-l1-1-0 00000001800094d4     ucrt:api-ms-win-crt-stdio-l1-1-0.dll
 0002:000034e8       __IMPORT_DESCRIPTOR_api-ms-win-crt-string-l1-1-0 00000001800094e8     ucrt:api-ms-win-crt-string-l1-1-0.dll
 0002:000034fc       __NULL_IMPORT_DESCRIPTOR   00000001800094fc     kernel32:KERNEL32.dll
 0003:00000060       _Init_global_epoch         000000018000a060     MSVCRT:thread_safe_statics.obj
 0003:00000070       __security_cookie          000000018000a070     MSVCRT:gs_cookie.obj
 0003:00000078       __security_cookie_complement 000000018000a078     MSVCRT:gs_cookie.obj
 0003:00000080       __scrt_native_dllmain_reason 000000018000a080     MSVCRT:utility.obj
 0003:00000088       __isa_available            000000018000a088     MSVCRT:cpu_disp.obj
 0003:0000008c       __isa_enabled              000000018000a08c     MSVCRT:cpu_disp.obj
 0003:00000090       __memset_fast_string_threshold 000000018000a090     MSVCRT:cpu_disp.obj
 0003:00000098       __memset_nt_threshold      000000018000a098     MSVCRT:cpu_disp.obj
 0003:000000a0       __scrt_ucrt_dll_is_in_use  000000018000a0a0     MSVCRT:ucrt_stubs.obj
 0003:000000b0       g_wrongHeapCallbacks       000000018000a0b0     libattach039Agent00.obj
 0003:00000130       g_szTagInfo                000000018000a130     libattach039Agent00.obj
 0003:00002070       g_tagFlags                 000000018000c070     libattach039Agent00.obj
 0003:00002458       g_refsToVerifyCnt          000000018000c458     libattach039Agent00.obj
 0003:0000245c       g_fakeUserData             000000018000c45c     libattach039Agent00.obj
 0003:00002460       g_tagVisitCount            000000018000c460     libattach039Agent00.obj
 0003:00003400       g_refsToVerify             000000018000d400     libattach039Agent00.obj
 0003:0001ab00       g_userDataError            0000000180024b00     libattach039Agent00.obj
 0003:0001ab04       threadStartReceived        0000000180024b04     libattach039Agent00.obj
 0003:0001ab08       threadWasExecuted          0000000180024b08     libattach039Agent00.obj
 0003:0001ab10       multiagentsOptions         0000000180024b10     libattach039Agent00.obj
 0003:0001ad70       ?_OptionsStorage@?1??__local_stdio_printf_options@@9@4_KA 0000000180024d70     libattach039Agent00.obj
 0003:0001b338       _tls_index                 0000000180025338     MSVCRT:tlssup.obj
 0003:0001b340       __scrt_current_native_startup_state 0000000180025340     MSVCRT:utility.obj
 0003:0001b348       __scrt_native_startup_lock 0000000180025348     MSVCRT:utility.obj
 0003:0001b388       __scrt_debugger_hook_flag  0000000180025388     MSVCRT:utility_desktop.obj
 0003:0001b390       ?__type_info_root_node@@3U__type_info_node@@A 0000000180025390     MSVCRT:tncleanup.obj
 0003:0001b3a0       ?_OptionsStorage@?1??__local_stdio_scanf_options@@9@4_KA 00000001800253a0     MSVCRT:default_local_stdio_options.obj
 0003:0001b3a8       __favor                    00000001800253a8     MSVCRT:cpu_disp.obj
 0003:0001b3b0       __dyn_tls_init_callback    00000001800253b0     <common>

 entry point at        0001:00003830

 Static symbols

 0000:fffd8000       .debug$S                   0000000180000000     attach039Agent00.exp
 0000:fffd8000       .debug$S                   0000000180000000     vcruntime:VCRUNTIME140.dll
 0000:fffd8000       .debug$S                   0000000180000000     vcruntime:VCRUNTIME140.dll
 0000:fffd8000       .debug$S                   0000000180000000     vcruntime:VCRUNTIME140.dll
 0000:fffd8000       .debug$S                   0000000180000000     vcruntime:VCRUNTIME140.dll
 0000:fffd8000       .debug$S                   0000000180000000     vcruntime:VCRUNTIME140.dll
 0000:fffd8000       .debug$S                   0000000180000000     vcruntime:VCRUNTIME140.dll
 0000:fffd8000       .debug$S                   0000000180000000     vcruntime:VCRUNTIME140.dll
 0000:fffd8000       .debug$S                   0000000180000000     ucrt:api-ms-win-crt-convert-l1-1-0.dll
 0002:ffffa000       .idata$6                   0000000180000000     ucrt:api-ms-win-crt-convert-l1-1-0.dll
 0000:fffd8000       .debug$S                   0000000180000000     ucrt:api-ms-win-crt-heap-l1-1-0.dll
 0000:fffd8000       .debug$S                   0000000180000000     ucrt:api-ms-win-crt-heap-l1-1-0.dll
 0000:fffd8000       .debug$S                   0000000180000000     ucrt:api-ms-win-crt-heap-l1-1-0.dll
 0000:fffd8000       .debug$S                   0000000180000000     ucrt:api-ms-win-crt-heap-l1-1-0.dll
 0000:fffd8000       .debug$S                   0000000180000000     ucrt:api-ms-win-crt-runtime-l1-1-0.dll
 0000:fffd8000       .debug$S                   0000000180000000     ucrt:api-ms-win-crt-runtime-l1-1-0.dll
 0000:fffd8000       .debug$S                   0000000180000000     ucrt:api-ms-win-crt-runtime-l1-1-0.dll
 0000:fffd8000       .debug$S                   0000000180000000     ucrt:api-ms-win-crt-runtime-l1-1-0.dll
 0000:fffd8000       .debug$S                   0000000180000000     ucrt:api-ms-win-crt-runtime-l1-1-0.dll
 0000:fffd8000       .debug$S                   0000000180000000     ucrt:api-ms-win-crt-runtime-l1-1-0.dll
 0000:fffd8000       .debug$S                   0000000180000000     ucrt:api-ms-win-crt-runtime-l1-1-0.dll
 0000:fffd8000       .debug$S                   0000000180000000     ucrt:api-ms-win-crt-runtime-l1-1-0.dll
 0000:fffd8000       .debug$S                   0000000180000000     ucrt:api-ms-win-crt-runtime-l1-1-0.dll
 0000:fffd8000       .debug$S                   0000000180000000     ucrt:api-ms-win-crt-runtime-l1-1-0.dll
 0000:fffd8000       .debug$S                   0000000180000000     ucrt:api-ms-win-crt-runtime-l1-1-0.dll
 0000:fffd8000       .debug$S                   0000000180000000     ucrt:api-ms-win-crt-runtime-l1-1-0.dll
 0000:fffd8000       .debug$S                   0000000180000000     ucrt:api-ms-win-crt-runtime-l1-1-0.dll
 0000:fffd8000       .debug$S                   0000000180000000     ucrt:api-ms-win-crt-runtime-l1-1-0.dll
 0000:fffd8000       .debug$S                   0000000180000000     ucrt:api-ms-win-crt-runtime-l1-1-0.dll
 0000:fffd8000       .debug$S                   0000000180000000     ucrt:api-ms-win-crt-runtime-l1-1-0.dll
 0000:fffd8000       .debug$S                   0000000180000000     ucrt:api-ms-win-crt-stdio-l1-1-0.dll
 0000:fffd8000       .debug$S                   0000000180000000     ucrt:api-ms-win-crt-stdio-l1-1-0.dll
 0000:fffd8000       .debug$S                   0000000180000000     ucrt:api-ms-win-crt-stdio-l1-1-0.dll
 0000:fffd8000       .debug$S                   0000000180000000     ucrt:api-ms-win-crt-stdio-l1-1-0.dll
 0000:fffd8000       .debug$S                   0000000180000000     ucrt:api-ms-win-crt-stdio-l1-1-0.dll
 0000:fffd8000       .debug$S                   0000000180000000     ucrt:api-ms-win-crt-stdio-l1-1-0.dll
 0000:fffd8000       .debug$S                   0000000180000000     ucrt:api-ms-win-crt-stdio-l1-1-0.dll
 0000:fffd8000       .debug$S                   0000000180000000     ucrt:api-ms-win-crt-stdio-l1-1-0.dll
 0000:fffd8000       .debug$S                   0000000180000000     ucrt:api-ms-win-crt-stdio-l1-1-0.dll
 0000:fffd8000       .debug$S                   0000000180000000     ucrt:api-ms-win-crt-stdio-l1-1-0.dll
 0000:fffd8000       .debug$S                   0000000180000000     ucrt:api-ms-win-crt-string-l1-1-0.dll
 0000:fffd8000       .debug$S                   0000000180000000     ucrt:api-ms-win-crt-string-l1-1-0.dll
 0000:fffd8000       .debug$S                   0000000180000000     ucrt:api-ms-win-crt-string-l1-1-0.dll
 0000:fffd8000       .debug$S                   0000000180000000     ucrt:api-ms-win-crt-string-l1-1-0.dll
 0000:fffd8000       .debug$S                   0000000180000000     ucrt:api-ms-win-crt-string-l1-1-0.dll
 0000:fffd8000       .debug$S                   0000000180000000     ucrt:api-ms-win-crt-string-l1-1-0.dll
 0000:fffd8000       .debug$S                   0000000180000000     ucrt:api-ms-win-crt-string-l1-1-0.dll
 0000:fffd8000       .debug$S                   0000000180000000     ucrt:api-ms-win-crt-string-l1-1-0.dll
 0000:fffd8000       .debug$S                   0000000180000000     ucrt:api-ms-win-crt-string-l1-1-0.dll
 0000:fffd8000       .debug$S                   0000000180000000     kernel32:KERNEL32.dll
 0000:fffd8000       .debug$S                   0000000180000000     kernel32:KERNEL32.dll
 0000:fffd8000       .debug$S                   0000000180000000     kernel32:KERNEL32.dll
 0000:fffd8000       .debug$S                   0000000180000000     kernel32:KERNEL32.dll
 0000:fffd8000       .debug$S                   0000000180000000     kernel32:KERNEL32.dll
 0000:fffd8000       .debug$S                   0000000180000000     kernel32:KERNEL32.dll
 0000:fffd8000       .debug$S                   0000000180000000     kernel32:KERNEL32.dll
 0000:fffd8000       .debug$S                   0000000180000000     kernel32:KERNEL32.dll
 0000:fffd8000       .debug$S                   0000000180000000     kernel32:KERNEL32.dll
 0000:fffd8000       .debug$S                   0000000180000000     kernel32:KERNEL32.dll
 0000:fffd8000       .debug$S                   0000000180000000     kernel32:KERNEL32.dll
 0000:fffd8000       .debug$S                   0000000180000000     kernel32:KERNEL32.dll
 0000:fffd8000       .debug$S                   0000000180000000     kernel32:KERNEL32.dll
 0000:fffd8000       .debug$S                   0000000180000000     kernel32:KERNEL32.dll
 0000:fffd8000       .debug$S                   0000000180000000     kernel32:KERNEL32.dll
 0000:fffd8000       .debug$S                   0000000180000000     kernel32:KERNEL32.dll
 0000:fffd8000       .debug$S                   0000000180000000     kernel32:KERNEL32.dll
 0000:fffd8000       .debug$S                   0000000180000000     kernel32:KERNEL32.dll
 0000:fffd8000       .debug$S                   0000000180000000     kernel32:KERNEL32.dll
 0000:fffd8000       .debug$S                   0000000180000000     kernel32:KERNEL32.dll
 0000:fffd8000       .debug$S                   0000000180000000     kernel32:KERNEL32.dll
 0000:fffd8000       .debug$S                   0000000180000000     kernel32:KERNEL32.dll
 0000:fffd8000       .debug$S                   0000000180000000     kernel32:KERNEL32.dll
 0000:fffd8000       .debug$S                   0000000180000000     kernel32:KERNEL32.dll
 0000:fffd8000       .debug$S                   0000000180000000     kernel32:KERNEL32.dll
 0000:fffd8000       .debug$S                   0000000180000000     kernel32:KERNEL32.dll
 0000:fffd8000       .debug$S                   0000000180000000     kernel32:KERNEL32.dll
 0000:fffd8000       .debug$S                   0000000180000000     kernel32:KERNEL32.dll
 0001:00000f48       addRefToVerify             0000000180001f48 f   libattach039Agent00.obj
 0001:00000fb4       agentThreadWrapper         0000000180001fb4 f   libattach039Agent00.obj
 0001:000011a4       file_basename              00000001800021a4 f   libattach039Agent00.obj
 0001:0000168c       nsk_aod_checkJNIException  000000018000268c f   libattach039Agent00.obj
 0001:00002950       startAgentThreadWrapper    0000000180003950 f   libattach039Agent00.obj
 0001:00002e70       syncDebuggeeStatus         0000000180003e70 f   libattach039Agent00.obj
 0001:000032f0       capture_previous_context   00000001800042f0 f   MSVCRT:gs_report.obj
 0001:00003364       ?__scrt_initialize_thread_safe_statics@@YAHXZ 0000000180004364 f   MSVCRT:thread_safe_statics.obj
 0001:00003434       ?__scrt_uninitialize_thread_safe_statics@@YAXXZ 0000000180004434 f   MSVCRT:thread_safe_statics.obj
 0001:000034e0       $$000000                   00000001800044e0     MSVCRT:amdsecgs.obj
 0001:00003510       ?dllmain_crt_dispatch@@YAHQEAUHINSTANCE__@@KQEAX@Z 0000000180004510 f   MSVCRT:dll_dllmain.obj
 0001:00003560       ?dllmain_crt_process_attach@@YAHQEAUHINSTANCE__@@QEAX@Z 0000000180004560 f   MSVCRT:dll_dllmain.obj
 0001:00003678       ?dllmain_crt_process_detach@@YAH_N@Z 0000000180004678 f   MSVCRT:dll_dllmain.obj
 0001:000036fc       ?dllmain_dispatch@@YAHQEAUHINSTANCE__@@KQEAX@Z 00000001800046fc f   MSVCRT:dll_dllmain.obj
 0001:00004120       $$000000                   0000000180005120     MSVCRT:guard_dispatch.obj
 0001:00004140       $$000000                   0000000180005140     MSVCRT:guard_xfg_dispatch.obj
 0001:00004156       ?fin$0@?0??dllmain_crt_process_attach@@YAHQEAUHINSTANCE__@@QEAX@Z@4HA 0000000180005156 f   MSVCRT:dll_dllmain.obj
 0001:0000416d       ?fin$0@?0??dllmain_crt_process_detach@@YAH_N@Z@4HA 000000018000516d f   MSVCRT:dll_dllmain.obj
 0001:00004186       ?fin$1@?0??dllmain_crt_process_detach@@YAH_N@Z@4HA 0000000180005186 f   MSVCRT:dll_dllmain.obj
 0001:0000419a       ?filt$0@?0??dllmain_dispatch@@YAHQEAUHINSTANCE__@@KQEAX@Z@4HA 000000018000519a f   MSVCRT:dll_dllmain.obj
 0001:000041d0       __scrt_is_nonwritable_in_current_image$filt$0 00000001800051d0 f   MSVCRT:utility.obj
 0002:00000208       ?__scrt_initialize_tss_var@@3P6AHXZEA 0000000180006208     MSVCRT:thread_safe_statics.obj
 0002:00000350       ?opcLengths@@3QBEB         0000000180006350     libattach039Agent00.obj
 0002:00002650       GS_ExceptionPointers       0000000180008650     MSVCRT:gs_report.obj
 0002:00002d38       $unwind$fprintf            0000000180008d38     libattach039Agent00.obj
 0002:00002d44       $unwind$printf             0000000180008d44     libattach039Agent00.obj
 0002:00002d50       $unwind$?CallStaticVoidMethod@JNIEnv_@@QEAAXPEAV_jclass@@PEAU_jmethodID@@ZZ 0000000180008d50     libattach039Agent00.obj
 0002:00002d50       $unwind$?NewObject@JNIEnv_@@QEAAPEAV_jobject@@PEAV_jclass@@PEAU_jmethodID@@ZZ 0000000180008d50     libattach039Agent00.obj
 0002:00002d50       $unwind$nsk_lcomplain      0000000180008d50     libattach039Agent00.obj
 0002:00002d50       $unwind$nsk_ldisplay       0000000180008d50     libattach039Agent00.obj
 0002:00002d58       $unwind$nsk_jvmti_aod_disableEventsAndFinish 0000000180008d58     libattach039Agent00.obj
 0002:00002d58       $unwind$nsk_lvdisplay      0000000180008d58     libattach039Agent00.obj
 0002:00002d58       $unwind$_RTC_Initialize    0000000180008d58     MSVCRT:initsect.obj
 0002:00002d58       $unwind$_RTC_Terminate     0000000180008d58     MSVCRT:initsect.obj
 0002:00002d58       $unwind$?__scrt_initialize_thread_safe_statics@@YAHXZ 0000000180008d58     MSVCRT:thread_safe_statics.obj
 0002:00002d64       $unwind$nsk_lvcomplain     0000000180008d64     libattach039Agent00.obj
 0002:00002d7c       $unwind$nsk_ltrace         0000000180008d7c     libattach039Agent00.obj
 0002:00002d7c       $unwind$__report_gsfailure 0000000180008d7c     MSVCRT:gs_report.obj
 0002:00002d84       $unwind$nsk_aod_checkJNIException 0000000180008d84     libattach039Agent00.obj
 0002:00002d84       $unwind$nsk_lvtrace        0000000180008d84     libattach039Agent00.obj
 0002:00002d84       $unwind$__raise_securityfailure 0000000180008d84     MSVCRT:gs_report.obj
 0002:00002d84       $unwind$__scrt_initialize_crt 0000000180008d84     MSVCRT:utility.obj
 0002:00002d84       $unwind$__scrt_initialize_onexit_tables 0000000180008d84     MSVCRT:utility.obj
 0002:00002d84       $unwind$__scrt_release_startup_lock 0000000180008d84     MSVCRT:utility.obj
 0002:00002d84       $unwind$__scrt_uninitialize_crt 0000000180008d84     MSVCRT:utility.obj
 0002:00002d84       $unwind$_onexit            0000000180008d84     MSVCRT:utility.obj
 0002:00002d8c       $unwind$nsk_lverify        0000000180008d8c     libattach039Agent00.obj
 0002:00002d9c       $unwind$nsk_vprintf        0000000180008d9c     libattach039Agent00.obj
 0002:00002dac       $unwind$nsk_printf         0000000180008dac     libattach039Agent00.obj
 0002:00002db4       $unwind$Agent_OnAttach     0000000180008db4     libattach039Agent00.obj
 0002:00002dd4       $unwind$?nsk_jni_lverify@@YAHHPEAUJNIEnv_@@HQEBDH1ZZ 0000000180008dd4     libattach039Agent00.obj
 0002:00002de8       $unwind$?nsk_jni_check_exception@@YAHPEAUJNIEnv_@@QEBDH@Z 0000000180008de8     libattach039Agent00.obj
 0002:00002e04       $unwind$nsk_jvmti_createJVMTIEnv 0000000180008e04     libattach039Agent00.obj
 0002:00002e18       $unwind$Java_nsk_jvmti_unit_FollowReferences_FollowRefObjects_resetTags 0000000180008e18     libattach039Agent00.obj
 0002:00002e18       $unwind$addRefToVerify     0000000180008e18     libattach039Agent00.obj
 0002:00002e18       $unwind$nsk_aod_internal_error 0000000180008e18     libattach039Agent00.obj
 0002:00002e18       $unwind$nsk_jvmti_resetAgentData 0000000180008e18     libattach039Agent00.obj
 0002:00002e18       $unwind$nsk_jvmti_setFailStatus 0000000180008e18     libattach039Agent00.obj
 0002:00002e18       $unwind$__scrt_initialize_default_local_stdio_options 0000000180008e18     MSVCRT:default_local_stdio_options.obj
 0002:00002e18       $unwind$?dllmain_crt_dispatch@@YAHQEAUHINSTANCE__@@KQEAX@Z 0000000180008e18     MSVCRT:dll_dllmain.obj
 0002:00002e18       $unwind$DllMain            0000000180008e18     MSVCRT:dll_dllmain_stub.obj
 0002:00002e18       $unwind$__GSHandlerCheck   0000000180008e18     MSVCRT:gshandler.obj
 0002:00002e18       $unwind$?__scrt_uninitialize_thread_safe_statics@@YAXXZ 0000000180008e18     MSVCRT:thread_safe_statics.obj
 0002:00002e18       $unwind$__scrt_acquire_startup_lock 0000000180008e18     MSVCRT:utility.obj
 0002:00002e18       $unwind$__scrt_dllmain_after_initialize_c 0000000180008e18     MSVCRT:utility.obj
 0002:00002e18       $unwind$__scrt_dllmain_before_initialize_c 0000000180008e18     MSVCRT:utility.obj
 0002:00002e18       $unwind$__scrt_dllmain_crt_thread_attach 0000000180008e18     MSVCRT:utility.obj
 0002:00002e18       $unwind$__scrt_dllmain_crt_thread_detach 0000000180008e18     MSVCRT:utility.obj
 0002:00002e18       $unwind$__scrt_dllmain_uninitialize_c 0000000180008e18     MSVCRT:utility.obj
 0002:00002e18       $unwind$__scrt_dllmain_uninitialize_critical 0000000180008e18     MSVCRT:utility.obj
 0002:00002e18       $unwind$atexit             0000000180008e18     MSVCRT:utility.obj
 0002:00002e20       $unwind$nsk_jvmti_lverify  0000000180008e20     libattach039Agent00.obj
 0002:00002e34       $unwind$exitOnError        0000000180008e34     libattach039Agent00.obj
 0002:00002e44       $unwind$Java_nsk_share_jvmti_ArgumentHandler_getAgentOptionsString 0000000180008e44     libattach039Agent00.obj
 0002:00002e44       $unwind$nsk_jvmti_aod_deallocate 0000000180008e44     libattach039Agent00.obj
 0002:00002e58       $unwind$Java_nsk_jvmti_unit_FollowReferences_FollowRefObjects_getTag 0000000180008e58     libattach039Agent00.obj
 0002:00002e58       $unwind$Java_nsk_share_jvmti_DebugeeClass_checkStatus 0000000180008e58     libattach039Agent00.obj
 0002:00002e58       $unwind$agentThreadWrapper 0000000180008e58     libattach039Agent00.obj
 0002:00002e68       $unwind$nsk_aod_agentLoaded 0000000180008e68     libattach039Agent00.obj
 0002:00002e68       $unwind$nsk_jvmti_aod_createThreadWithName 0000000180008e68     libattach039Agent00.obj
 0002:00002e68       $unwind$startAgentThreadWrapper 0000000180008e68     libattach039Agent00.obj
 0002:00002e84       $unwind$syncDebuggeeStatus 0000000180008e84     libattach039Agent00.obj
 0002:00002e84       $unwind$__scrt_dllmain_exception_filter 0000000180008e84     MSVCRT:utility.obj
 0002:00002e98       $unwind$Java_nsk_share_jvmti_DebugeeClass_resetAgentData 0000000180008e98     libattach039Agent00.obj
 0002:00002e98       $unwind$nsk_aod_createJNIEnv 0000000180008e98     libattach039Agent00.obj
 0002:00002ea0       $unwind$MA_checkStatus     0000000180008ea0     libattach039Agent00.obj
 0002:00002eb4       $unwind$Java_nsk_jvmti_unit_FollowReferences_FollowRefObjects_setTag 0000000180008eb4     libattach039Agent00.obj
 0002:00002ecc       $unwind$Java_nsk_jvmti_unit_FollowReferences_FollowRefObjects_addRefToVerify 0000000180008ecc     libattach039Agent00.obj
 0002:00002ee8       $unwind$nsk_aod_createOptions 0000000180008ee8     libattach039Agent00.obj
 0002:00002f04       $unwind$nsk_aod_getOptionValue 0000000180008f04     libattach039Agent00.obj
 0002:00002f04       $unwind$nsk_aod_optionSpecified 0000000180008f04     libattach039Agent00.obj
 0002:00002f18       $unwind$nsk_aod_agentFinished 0000000180008f18     libattach039Agent00.obj
 0002:00002f30       $unwind$nsk_free_options   0000000180008f30     libattach039Agent00.obj
 0002:00002f40       $unwind$nsk_jvmti_aod_getThreadName 0000000180008f40     libattach039Agent00.obj
 0002:00002f58       $unwind$nsk_jvmti_aod_enableEvents 0000000180008f58     libattach039Agent00.obj
 0002:00002f70       $unwind$nsk_jvmti_aod_disableEvents 0000000180008f70     libattach039Agent00.obj
 0002:00002f88       $unwind$startedThreadFunction 0000000180008f88     libattach039Agent00.obj
 0002:00002fa0       $unwind$startNewThread     0000000180008fa0     libattach039Agent00.obj
 0002:00002fb8       $unwind$threadEndHandler   0000000180008fb8     libattach039Agent00.obj
 0002:00002fb8       $unwind$threadStartHandler 0000000180008fb8     libattach039Agent00.obj
 0002:00002fd0       $unwind$capture_previous_context 0000000180008fd0     MSVCRT:gs_report.obj
 0002:00002fdc       $unwind$__GSHandlerCheckCommon 0000000180008fdc     MSVCRT:gshandler.obj
 0002:00002fe8       $xdatasym                  0000000180008fe8     MSVCRT:amdsecgs.obj
 0002:00002fec       $unwind$?dllmain_crt_process_attach@@YAHQEAUHINSTANCE__@@QEAX@Z 0000000180008fec     MSVCRT:dll_dllmain.obj
 0002:00003028       $unwind$?fin$0@?0??dllmain_crt_process_attach@@YAHQEAUHINSTANCE__@@QEAX@Z@4HA 0000000180009028     MSVCRT:dll_dllmain.obj
 0002:00003028       $unwind$?fin$0@?0??dllmain_crt_process_detach@@YAH_N@Z@4HA 0000000180009028     MSVCRT:dll_dllmain.obj
 0002:00003028       $unwind$?fin$1@?0??dllmain_crt_process_detach@@YAH_N@Z@4HA 0000000180009028     MSVCRT:dll_dllmain.obj
 0002:00003030       $unwind$?dllmain_crt_process_detach@@YAH_N@Z 0000000180009030     MSVCRT:dll_dllmain.obj
 0002:00003084       $unwind$?dllmain_dispatch@@YAHQEAUHINSTANCE__@@KQEAX@Z 0000000180009084     MSVCRT:dll_dllmain.obj
 0002:000030ac       $unwind$?filt$0@?0??dllmain_dispatch@@YAHQEAUHINSTANCE__@@KQEAX@Z@4HA 00000001800090ac     MSVCRT:dll_dllmain.obj
 0002:000030b4       $unwind$_DllMainCRTStartup 00000001800090b4     MSVCRT:dll_dllmain.obj
 0002:000030c4       $unwind$__scrt_is_nonwritable_in_current_image 00000001800090c4     MSVCRT:utility.obj
 0002:000030e4       $unwind$__scrt_is_nonwritable_in_current_image$filt$0 00000001800090e4     MSVCRT:utility.obj
 0002:000030ec       $unwind$__scrt_fastfail    00000001800090ec     MSVCRT:utility_desktop.obj
 0002:000030fc       $unwind$__security_init_cookie 00000001800090fc     MSVCRT:gs_support.obj
 0002:00003108       $unwind$__isa_available_init 0000000180009108     MSVCRT:cpu_disp.obj
 0002:00003118       $xdatasym                  0000000180009118     MSVCRT:guard_dispatch.obj
 0002:00003120       $xdatasym                  0000000180009120     MSVCRT:guard_xfg_dispatch.obj
 0002:00003130       .edata                     0000000180009130     attach039Agent00.exp
 0002:00003158       rgpv                       0000000180009158     attach039Agent00.exp
 0002:0000318c       rgszName                   000000018000918c     attach039Agent00.exp
 0002:000031c0       rgwOrd                     00000001800091c0     attach039Agent00.exp
 0002:000031da       szName                     00000001800091da     attach039Agent00.exp
 0002:000031ef       $N00001                    00000001800091ef     attach039Agent00.exp
 0002:000031fe       $N00002                    00000001800091fe     attach039Agent00.exp
 0002:00003243       $N00003                    0000000180009243     attach039Agent00.exp
 0002:00003280       $N00004                    0000000180009280     attach039Agent00.exp
 0002:000032c8       $N00005                    00000001800092c8     attach039Agent00.exp
 0002:00003308       $N00006                    0000000180009308     attach039Agent00.exp
 0002:00003345       $N00007                    0000000180009345     attach039Agent00.exp
 0002:00003380       $N00008                    0000000180009380     attach039Agent00.exp
 0002:000033ae       $N00009                    00000001800093ae     attach039Agent00.exp
 0002:000033df       $N00010                    00000001800093df     attach039Agent00.exp
 0002:0000340e       $N00011                    000000018000940e     attach039Agent00.exp
 0002:0000343d       $N00012                    000000018000943d     attach039Agent00.exp
 0002:00003472       $N00013                    0000000180009472     attach039Agent00.exp
 0002:000038b2       .idata$6                   00000001800098b2     kernel32:KERNEL32.dll
 0002:00003916       .idata$6                   0000000180009916     vcruntime:VCRUNTIME140.dll
 0002:00003a9e       .idata$6                   0000000180009a9e     ucrt:api-ms-win-crt-heap-l1-1-0.dll
 0002:00003abe       .idata$6                   0000000180009abe     ucrt:api-ms-win-crt-runtime-l1-1-0.dll
 0002:00003ae0       .idata$6                   0000000180009ae0     ucrt:api-ms-win-crt-stdio-l1-1-0.dll
 0002:00003b00       .idata$6                   0000000180009b00     ucrt:api-ms-win-crt-string-l1-1-0.dll
 0003:00000000       ?codeAttributeName@@3PEBDEB 000000018000a000     libattach039Agent00.obj
 0003:00000008       ?lineNumberAttributeName@@3PEBDEB 000000018000a008     libattach039Agent00.obj
 0003:00000010       ?localVarAttributeName@@3PEBDEB 000000018000a010     libattach039Agent00.obj
 0003:00000018       ?localVarTypeAttributeName@@3PEBDEB 000000018000a018     libattach039Agent00.obj
 0003:00000020       ?stackMapAttributeName@@3PEBDEB 000000018000a020     libattach039Agent00.obj
 0003:00000028       ?callBytes@@3PAEA          000000018000a028     libattach039Agent00.obj
 0003:0000002c       ?allocBytes@@3PAEA         000000018000a02c     libattach039Agent00.obj
 0003:00000030       TARGET_APP_CLASS_NAME      000000018000a030     libattach039Agent00.obj
 0003:00000038       AGENT_LOADED_METHOD_NAME   000000018000a038     libattach039Agent00.obj
 0003:00000040       AGENT_LOADED_METHOD_SIGNATURE 000000018000a040     libattach039Agent00.obj
 0003:00000048       AGENT_FINISHED_METHOD_NAME 000000018000a048     libattach039Agent00.obj
 0003:00000050       AGENT_FINISHED_METHOD_SIGNATURE 000000018000a050     libattach039Agent00.obj
 0003:00000058       testEvents                 000000018000a058     libattach039Agent00.obj
 0003:0001abb0       nsk_context                0000000180024bb0     libattach039Agent00.obj
 0003:0001abbc       redefineAttempted          0000000180024bbc     libattach039Agent00.obj
 0003:0001abc0       redefineSucceed            0000000180024bc0     libattach039Agent00.obj
 0003:0001abc4       agentFailed                0000000180024bc4     libattach039Agent00.obj
 0003:0001abc8       agentThread                0000000180024bc8     libattach039Agent00.obj
 0003:0001abd0       context                    0000000180024bd0     libattach039Agent00.obj
 0003:0001ac88       agentThreadProc            0000000180024c88     libattach039Agent00.obj
 0003:0001ac90       agentThreadArg             0000000180024c90     libattach039Agent00.obj
 0003:0001ac98       agent_data                 0000000180024c98     libattach039Agent00.obj
 0003:0001aca8       jvmti_env                  0000000180024ca8     libattach039Agent00.obj
 0003:0001acb0       jvm                        0000000180024cb0     libattach039Agent00.obj
 0003:0001acb8       jni_env                    0000000180024cb8     libattach039Agent00.obj
 0003:0001acc0       currentAgentStatus         0000000180024cc0     libattach039Agent00.obj
 0003:0001acc4       ?codeAttributeIndex@@3GA   0000000180024cc4     libattach039Agent00.obj
 0003:0001acc8       checkStatus_func           0000000180024cc8     libattach039Agent00.obj
 0003:0001acd0       ?lineNumberAttributeIndex@@3GA 0000000180024cd0     libattach039Agent00.obj
 0003:0001acd4       ?localVarAttributeIndex@@3GA 0000000180024cd4     libattach039Agent00.obj
 0003:0001acd8       ?localVarTypeAttributeIndex@@3GA 0000000180024cd8     libattach039Agent00.obj
 0003:0001acdc       ?stackMapAttributeIndex@@3GA 0000000180024cdc     libattach039Agent00.obj
 0003:0001ace0       ?stackFrameOffset@@3GA     0000000180024ce0     libattach039Agent00.obj
 0003:0001ace4       ?mode@@3HA                 0000000180024ce4     libattach039Agent00.obj
 0003:0001ace8       ?orig@@3PEBEEB             0000000180024ce8     libattach039Agent00.obj
 0003:0001acf0       ?gen@@3PEAEEA              0000000180024cf0     libattach039Agent00.obj
 0003:0001acf8       ?inputPos@@3PEAEEA         0000000180024cf8     libattach039Agent00.obj
 0003:0001ad00       ?endPos@@3PEBEEB           0000000180024d00     libattach039Agent00.obj
 0003:0001ad08       ?genPos@@3PEAEEA           0000000180024d08     libattach039Agent00.obj
 0003:0001ad10       ?markPos@@3PEAEEA          0000000180024d10     libattach039Agent00.obj
 0003:0001ad18       ?constantPool@@3PEAPEADEA  0000000180024d18     libattach039Agent00.obj
 0003:0001ad20       ?constantPoolSize@@3GA     0000000180024d20     libattach039Agent00.obj
 0003:0001ad24       ?constantPoolCount@@3GA    0000000180024d24     libattach039Agent00.obj
 0003:0001ad28       ?zeroBytes@@3PAEA          0000000180024d28     libattach039Agent00.obj
 0003:0001ad2c       ?codeLength@@3IA           0000000180024d2c     libattach039Agent00.obj
 0003:0001ad30       ?map@@3PEAIEA              0000000180024d30     libattach039Agent00.obj
 0003:0001ad38       ?widening@@3PEACEA         0000000180024d38     libattach039Agent00.obj
 0003:0001ad40       internalError              0000000180024d40     libattach039Agent00.obj
 0003:0001ad44       multiagentsCount           0000000180024d44     libattach039Agent00.obj
 0003:0001ad48       targetAppClass             0000000180024d48     libattach039Agent00.obj
 0003:0001ad50       agentLoadedMethod          0000000180024d50     libattach039Agent00.obj
 0003:0001ad58       agentFinishedMethod        0000000180024d58     libattach039Agent00.obj
 0003:0001ad60       options                    0000000180024d60     libattach039Agent00.obj
 0003:0001ad68       agentName                  0000000180024d68     libattach039Agent00.obj
 0003:0001ad80       GS_ExceptionRecord         0000000180024d80     MSVCRT:gs_report.obj
 0003:0001ae20       GS_ContextRecord           0000000180024e20     MSVCRT:gs_report.obj
 0003:0001b2f0       ?g_tss_cv@@3U_RTL_CONDITION_VARIABLE@@A 00000001800252f0     MSVCRT:thread_safe_statics.obj
 0003:0001b2f8       ?g_tss_event@@3PEAXEA      00000001800252f8     MSVCRT:thread_safe_statics.obj
 0003:0001b300       ?g_tss_mutex@@3U_RTL_CRITICAL_SECTION@@A 0000000180025300     MSVCRT:thread_safe_statics.obj
 0003:0001b328       ?g_sleep_condition_variable_cs@@3P6AHPEAU_RTL_CONDITION_VARIABLE@@PEAU_RTL_CRITICAL_SECTION@@K@ZEA 0000000180025328     MSVCRT:thread_safe_statics.obj
 0003:0001b330       ?g_wake_all_condition_variable@@3P6AXPEAU_RTL_CONDITION_VARIABLE@@@ZEA 0000000180025330     MSVCRT:thread_safe_statics.obj
 0003:0001b33c       ?__proc_attached@@3HA      000000018002533c     MSVCRT:dll_dllmain.obj
 0003:0001b350       ?is_initialized_as_dll@@3_NA 0000000180025350     MSVCRT:utility.obj
 0003:0001b351       ?module_local_atexit_table_initialized@@3_NA 0000000180025351     MSVCRT:utility.obj
 0003:0001b358       ?module_local_atexit_table@@3U_onexit_table_t@@A 0000000180025358     MSVCRT:utility.obj
 0003:0001b370       ?module_local_at_quick_exit_table@@3U_onexit_table_t@@A 0000000180025370     MSVCRT:utility.obj
